 windowsaccessbridge-64

 Timestamp is 3e31843c (reproducible build file hash)

 Preferred load address is 0000000180000000

 Start         Length     Name                   Class
 0001:00000000 000075d0H .text$mn                CODE
 0001:000075d0 00000036H .text$mn$00             CODE
 0001:00007606 00000092H .text$x                 CODE
 0002:00000000 00000228H .idata$5                DATA
 0002:00000228 00000038H .00cfg                  DATA
 0002:00000260 00000008H .CRT$XCA                DATA
 0002:00000268 00000008H .CRT$XCZ                DATA
 0002:00000270 00000008H .CRT$XIA                DATA
 0002:00000278 00000008H .CRT$XIZ                DATA
 0002:00000280 00000008H .CRT$XPA                DATA
 0002:00000288 00000008H .CRT$XPZ                DATA
 0002:00000290 00000008H .CRT$XTA                DATA
 0002:00000298 00000008H .CRT$XTZ                DATA
 0002:000002a0 00000000H .gehcont$y              DATA
 0002:000002a0 00000000H .gfids$y                DATA
 0002:000002a0 00003860H .rdata                  DATA
 0002:00003b00 00000000H .rdata$CastGuardVftablesA DATA
 0002:00003b00 00000000H .rdata$CastGuardVftablesC DATA
 0002:00003b00 000001f4H .rdata$r                DATA
 0002:00003cf4 0000006cH .rdata$voltmd           DATA
 0002:00003d60 00000318H .rdata$zzzdbg           DATA
 0002:00004078 00000008H .rtc$IAA                DATA
 0002:00004080 00000008H .rtc$IZZ                DATA
 0002:00004088 00000008H .rtc$TAA                DATA
 0002:00004090 00000008H .rtc$TZZ                DATA
 0002:00004098 00000618H .xdata                  DATA
 0002:000046b0 000000f0H .xdata$x                DATA
 0002:000047a0 00000da0H .edata                  DATA
 0002:00005540 000000a0H .idata$2                DATA
 0002:000055e0 00000018H .idata$3                DATA
 0002:000055f8 00000228H .idata$4                DATA
 0002:00005820 0000055cH .idata$6                DATA
 0003:00000000 00000038H .data                   DATA
 0003:00000038 00000080H .data$r                 DATA
 0003:000000b8 00000028H .data$rs                DATA
 0003:000000e0 00000640H .bss                    DATA
 0004:00000000 00000aecH .pdata                  DATA
 0005:00000000 00000120H .rsrc$01                DATA
 0005:00000120 000006b8H .rsrc$02                DATA

  Address         Publics by Value              Rva+Base               Lib:Object

 0000:00000000       __AbsoluteZero             0000000000000000     <absolute>
 0000:00000000       ___safe_se_handler_count   0000000000000000     <absolute>
 0000:00000000       ___safe_se_handler_table   0000000000000000     <absolute>
 0000:00000000       __arm64x_extra_rfe_table   0000000000000000     <absolute>
 0000:00000000       __arm64x_extra_rfe_table_size 0000000000000000     <absolute>
 0000:00000000       __arm64x_native_entrypoint 0000000000000000     <absolute>
 0000:00000000       __arm64x_redirection_metadata 0000000000000000     <absolute>
 0000:00000000       __arm64x_redirection_metadata_count 0000000000000000     <absolute>
 0000:00000000       __dynamic_value_reloc_table 0000000000000000     <absolute>
 0000:00000000       __enclave_config           0000000000000000     <absolute>
 0000:00000000       __guard_check_icall_a64n_fptr 0000000000000000     <absolute>
 0000:00000000       __guard_eh_cont_count      0000000000000000     <absolute>
 0000:00000000       __guard_eh_cont_table      0000000000000000     <absolute>
 0000:00000000       __guard_fids_count         0000000000000000     <absolute>
 0000:00000000       __guard_fids_table         0000000000000000     <absolute>
 0000:00000000       __guard_iat_count          0000000000000000     <absolute>
 0000:00000000       __guard_iat_table          0000000000000000     <absolute>
 0000:00000000       __guard_longjmp_count      0000000000000000     <absolute>
 0000:00000000       __guard_longjmp_table      0000000000000000     <absolute>
 0000:00000000       __hybrid_auxiliary_iat     0000000000000000     <absolute>
 0000:00000000       __hybrid_auxiliary_iat_copy 0000000000000000     <absolute>
 0000:00000000       __hybrid_code_map          0000000000000000     <absolute>
 0000:00000000       __hybrid_code_map_count    0000000000000000     <absolute>
 0000:00000000       __x64_code_ranges_to_entry_points 0000000000000000     <absolute>
 0000:00000000       __x64_code_ranges_to_entry_points_count 0000000000000000     <absolute>
 0000:00000100       __guard_flags              0000000000000100     <absolute>
 0000:00000000       __ImageBase                0000000180000000     <linker-defined>
 0001:00000000       PrintDebugString           0000000180001000 f   AccessBridgeDebug.obj
 0001:00000080       __local_stdio_printf_options 0000000180001080 f i AccessBridgeDebug.obj
 0001:00000088       finalizeFileLogger         0000000180001088 f   AccessBridgeDebug.obj
 0001:000000ac       fprintf                    00000001800010ac f i AccessBridgeDebug.obj
 0001:000000f0       getTimeStamp               00000001800010f0 f   AccessBridgeDebug.obj
 0001:00000128       initializeFileLogger       0000000180001128 f   AccessBridgeDebug.obj
 0001:00000238       printf                     0000000180001238 f i AccessBridgeDebug.obj
 0001:00000288       ??0AccessBridgeEventHandler@@QEAA@XZ 0000000180001288 f   AccessBridgeEventHandler.obj
 0001:00000324       ??1AccessBridgeEventHandler@@QEAA@XZ 0000000180001324 f   AccessBridgeEventHandler.obj
 0001:00000324       ??1AccessBridgeMessageQueue@@QEAA@XZ 0000000180001324 f   AccessBridgeMessageQueue.obj
 0001:00000324       _guard_check_icall_nop     0000000180001324 f   MSVCRT:guard_support.obj
 0001:00000328       ?fireCaretUpdate@AccessBridgeEventHandler@@QEAAXJ_J0@Z 0000000180001328 f   AccessBridgeEventHandler.obj
 0001:0000034c       ?fireFocusGained@AccessBridgeEventHandler@@QEAAXJ_J0@Z 000000018000134c f   AccessBridgeEventHandler.obj
 0001:00000370       ?fireFocusLost@AccessBridgeEventHandler@@QEAAXJ_J0@Z 0000000180001370 f   AccessBridgeEventHandler.obj
 0001:00000394       ?fireJavaShutdown@AccessBridgeEventHandler@@QEAAXJ@Z 0000000180001394 f   AccessBridgeEventHandler.obj
 0001:000003ac       ?fireMenuCanceled@AccessBridgeEventHandler@@QEAAXJ_J0@Z 00000001800013ac f   AccessBridgeEventHandler.obj
 0001:000003d0       ?fireMenuDeselected@AccessBridgeEventHandler@@QEAAXJ_J0@Z 00000001800013d0 f   AccessBridgeEventHandler.obj
 0001:000003f4       ?fireMenuSelected@AccessBridgeEventHandler@@QEAAXJ_J0@Z 00000001800013f4 f   AccessBridgeEventHandler.obj
 0001:00000418       ?fireMouseClicked@AccessBridgeEventHandler@@QEAAXJ_J0@Z 0000000180001418 f   AccessBridgeEventHandler.obj
 0001:0000043c       ?fireMouseEntered@AccessBridgeEventHandler@@QEAAXJ_J0@Z 000000018000143c f   AccessBridgeEventHandler.obj
 0001:00000460       ?fireMouseExited@AccessBridgeEventHandler@@QEAAXJ_J0@Z 0000000180001460 f   AccessBridgeEventHandler.obj
 0001:00000484       ?fireMousePressed@AccessBridgeEventHandler@@QEAAXJ_J0@Z 0000000180001484 f   AccessBridgeEventHandler.obj
 0001:000004a8       ?fireMouseReleased@AccessBridgeEventHandler@@QEAAXJ_J0@Z 00000001800014a8 f   AccessBridgeEventHandler.obj
 0001:000004cc       ?firePopupMenuCanceled@AccessBridgeEventHandler@@QEAAXJ_J0@Z 00000001800014cc f   AccessBridgeEventHandler.obj
 0001:000004f0       ?firePopupMenuWillBecomeInvisible@AccessBridgeEventHandler@@QEAAXJ_J0@Z 00000001800014f0 f   AccessBridgeEventHandler.obj
 0001:00000514       ?firePopupMenuWillBecomeVisible@AccessBridgeEventHandler@@QEAAXJ_J0@Z 0000000180001514 f   AccessBridgeEventHandler.obj
 0001:0000053c       ?firePropertyActiveDescendentChange@AccessBridgeEventHandler@@QEAAXJ_J000@Z 000000018000153c f   AccessBridgeEventHandler.obj
 0001:00000580       ?firePropertyCaretChange@AccessBridgeEventHandler@@QEAAXJ_J0HH@Z 0000000180001580 f   AccessBridgeEventHandler.obj
 0001:000005c4       ?firePropertyChildChange@AccessBridgeEventHandler@@QEAAXJ_J000@Z 00000001800015c4 f   AccessBridgeEventHandler.obj
 0001:00000608       ?firePropertyDescriptionChange@AccessBridgeEventHandler@@QEAAXJ_J0PEAG1@Z 0000000180001608 f   AccessBridgeEventHandler.obj
 0001:0000064c       ?firePropertyNameChange@AccessBridgeEventHandler@@QEAAXJ_J0PEAG1@Z 000000018000164c f   AccessBridgeEventHandler.obj
 0001:00000690       ?firePropertySelectionChange@AccessBridgeEventHandler@@QEAAXJ_J0@Z 0000000180001690 f   AccessBridgeEventHandler.obj
 0001:000006b8       ?firePropertyStateChange@AccessBridgeEventHandler@@QEAAXJ_J0PEAG1@Z 00000001800016b8 f   AccessBridgeEventHandler.obj
 0001:000006fc       ?firePropertyTableModelChange@AccessBridgeEventHandler@@QEAAXJ_J0PEAG1@Z 00000001800016fc f   AccessBridgeEventHandler.obj
 0001:00000740       ?firePropertyTextChange@AccessBridgeEventHandler@@QEAAXJ_J0@Z 0000000180001740 f   AccessBridgeEventHandler.obj
 0001:00000768       ?firePropertyValueChange@AccessBridgeEventHandler@@QEAAXJ_J0PEAG1@Z 0000000180001768 f   AccessBridgeEventHandler.obj
 0001:000007ac       ?firePropertyVisibleDataChange@AccessBridgeEventHandler@@QEAAXJ_J0@Z 00000001800017ac f   AccessBridgeEventHandler.obj
 0001:000007d4       ?setCaretUpdateFP@AccessBridgeEventHandler@@QEAAXP6AXJ_J0@ZPEAVWinAccessBridge@@@Z 00000001800017d4 f   AccessBridgeEventHandler.obj
 0001:00000800       ?setFocusGainedFP@AccessBridgeEventHandler@@QEAAXP6AXJ_J0@ZPEAVWinAccessBridge@@@Z 0000000180001800 f   AccessBridgeEventHandler.obj
 0001:0000082c       ?setFocusLostFP@AccessBridgeEventHandler@@QEAAXP6AXJ_J0@ZPEAVWinAccessBridge@@@Z 000000018000182c f   AccessBridgeEventHandler.obj
 0001:00000858       ?setJavaShutdownFP@AccessBridgeEventHandler@@QEAAXP6AXJ@ZPEAVWinAccessBridge@@@Z 0000000180001858 f   AccessBridgeEventHandler.obj
 0001:00000884       ?setMenuCanceledFP@AccessBridgeEventHandler@@QEAAXP6AXJ_J0@ZPEAVWinAccessBridge@@@Z 0000000180001884 f   AccessBridgeEventHandler.obj
 0001:000008b0       ?setMenuDeselectedFP@AccessBridgeEventHandler@@QEAAXP6AXJ_J0@ZPEAVWinAccessBridge@@@Z 00000001800018b0 f   AccessBridgeEventHandler.obj
 0001:000008dc       ?setMenuSelectedFP@AccessBridgeEventHandler@@QEAAXP6AXJ_J0@ZPEAVWinAccessBridge@@@Z 00000001800018dc f   AccessBridgeEventHandler.obj
 0001:00000908       ?setMouseClickedFP@AccessBridgeEventHandler@@QEAAXP6AXJ_J0@ZPEAVWinAccessBridge@@@Z 0000000180001908 f   AccessBridgeEventHandler.obj
 0001:00000934       ?setMouseEnteredFP@AccessBridgeEventHandler@@QEAAXP6AXJ_J0@ZPEAVWinAccessBridge@@@Z 0000000180001934 f   AccessBridgeEventHandler.obj
 0001:00000960       ?setMouseExitedFP@AccessBridgeEventHandler@@QEAAXP6AXJ_J0@ZPEAVWinAccessBridge@@@Z 0000000180001960 f   AccessBridgeEventHandler.obj
 0001:0000098c       ?setMousePressedFP@AccessBridgeEventHandler@@QEAAXP6AXJ_J0@ZPEAVWinAccessBridge@@@Z 000000018000198c f   AccessBridgeEventHandler.obj
 0001:000009b8       ?setMouseReleasedFP@AccessBridgeEventHandler@@QEAAXP6AXJ_J0@ZPEAVWinAccessBridge@@@Z 00000001800019b8 f   AccessBridgeEventHandler.obj
 0001:000009e4       ?setPopupMenuCanceledFP@AccessBridgeEventHandler@@QEAAXP6AXJ_J0@ZPEAVWinAccessBridge@@@Z 00000001800019e4 f   AccessBridgeEventHandler.obj
 0001:00000a10       ?setPopupMenuWillBecomeInvisibleFP@AccessBridgeEventHandler@@QEAAXP6AXJ_J0@ZPEAVWinAccessBridge@@@Z 0000000180001a10 f   AccessBridgeEventHandler.obj
 0001:00000a3c       ?setPopupMenuWillBecomeVisibleFP@AccessBridgeEventHandler@@QEAAXP6AXJ_J0@ZPEAVWinAccessBridge@@@Z 0000000180001a3c f   AccessBridgeEventHandler.obj
 0001:00000a6c       ?setPropertyActiveDescendentChangeFP@AccessBridgeEventHandler@@QEAAXP6AXJ_J000@ZPEAVWinAccessBridge@@@Z 0000000180001a6c f   AccessBridgeEventHandler.obj
 0001:00000a9c       ?setPropertyCaretChangeFP@AccessBridgeEventHandler@@QEAAXP6AXJ_J0HH@ZPEAVWinAccessBridge@@@Z 0000000180001a9c f   AccessBridgeEventHandler.obj
 0001:00000acc       ?setPropertyChangeFP@AccessBridgeEventHandler@@QEAAXP6AXJ_J0PEAG11@ZPEAVWinAccessBridge@@@Z 0000000180001acc f   AccessBridgeEventHandler.obj
 0001:00000af8       ?setPropertyChildChangeFP@AccessBridgeEventHandler@@QEAAXP6AXJ_J000@ZPEAVWinAccessBridge@@@Z 0000000180001af8 f   AccessBridgeEventHandler.obj
 0001:00000b28       ?setPropertyDescriptionChangeFP@AccessBridgeEventHandler@@QEAAXP6AXJ_J0PEAG1@ZPEAVWinAccessBridge@@@Z 0000000180001b28 f   AccessBridgeEventHandler.obj
 0001:00000b58       ?setPropertyNameChangeFP@AccessBridgeEventHandler@@QEAAXP6AXJ_J0PEAG1@ZPEAVWinAccessBridge@@@Z 0000000180001b58 f   AccessBridgeEventHandler.obj
 0001:00000b88       ?setPropertySelectionChangeFP@AccessBridgeEventHandler@@QEAAXP6AXJ_J0@ZPEAVWinAccessBridge@@@Z 0000000180001b88 f   AccessBridgeEventHandler.obj
 0001:00000bb8       ?setPropertyStateChangeFP@AccessBridgeEventHandler@@QEAAXP6AXJ_J0PEAG1@ZPEAVWinAccessBridge@@@Z 0000000180001bb8 f   AccessBridgeEventHandler.obj
 0001:00000be8       ?setPropertyTableModelChangeFP@AccessBridgeEventHandler@@QEAAXP6AXJ_J0PEAG1@ZPEAVWinAccessBridge@@@Z 0000000180001be8 f   AccessBridgeEventHandler.obj
 0001:00000c18       ?setPropertyTextChangeFP@AccessBridgeEventHandler@@QEAAXP6AXJ_J0@ZPEAVWinAccessBridge@@@Z 0000000180001c18 f   AccessBridgeEventHandler.obj
 0001:00000c48       ?setPropertyValueChangeFP@AccessBridgeEventHandler@@QEAAXP6AXJ_J0PEAG1@ZPEAVWinAccessBridge@@@Z 0000000180001c48 f   AccessBridgeEventHandler.obj
 0001:00000c78       ?setPropertyVisibleDataChangeFP@AccessBridgeEventHandler@@QEAAXP6AXJ_J0@ZPEAVWinAccessBridge@@@Z 0000000180001c78 f   AccessBridgeEventHandler.obj
 0001:00000ca8       ??0AccessBridgeJavaVMInstance@@QEAA@PEAUHWND__@@0JPEAV0@@Z 0000000180001ca8 f   AccessBridgeJavaVMInstance.obj
 0001:00000cfc       ??1AccessBridgeJavaVMInstance@@QEAA@XZ 0000000180001cfc f   AccessBridgeJavaVMInstance.obj
 0001:00000d58       ?findABJavaVMInstanceFromJavaHWND@AccessBridgeJavaVMInstance@@QEAAPEAV1@PEAUHWND__@@@Z 0000000180001d58 f   AccessBridgeJavaVMInstance.obj
 0001:00000dac       ?findAccessBridgeWindow@AccessBridgeJavaVMInstance@@QEAAPEAUHWND__@@J@Z 0000000180001dac f   AccessBridgeJavaVMInstance.obj
 0001:00000e0c       ?initiateIPC@AccessBridgeJavaVMInstance@@QEAA_JXZ 0000000180001e0c f   AccessBridgeJavaVMInstance.obj
 0001:00000f04       ?sendMemoryPackage@AccessBridgeJavaVMInstance@@QEAAHPEADJ@Z 0000000180001f04 f   AccessBridgeJavaVMInstance.obj
 0001:00000ff8       ?sendPackage@AccessBridgeJavaVMInstance@@QEAA_JPEADJ@Z 0000000180001ff8 f   AccessBridgeJavaVMInstance.obj
 0001:00001068       snprintf                   0000000180002068 f i AccessBridgeJavaVMInstance.obj
 0001:000010c0       ??0AccessBridgeMessageQueue@@QEAA@XZ 00000001800020c0 f   AccessBridgeMessageQueue.obj
 0001:000010d4       ??0AccessBridgeQueueElement@@QEAA@PEADH@Z 00000001800020d4 f   AccessBridgeMessageQueue.obj
 0001:0000113c       ??0bad_alloc@std@@QEAA@AEBV01@@Z 000000018000213c f i AccessBridgeMessageQueue.obj
 0001:00001178       ??0bad_alloc@std@@QEAA@XZ  0000000180002178 f i AccessBridgeMessageQueue.obj
 0001:00001198       ??0exception@std@@QEAA@AEBV01@@Z 0000000180002198 f i AccessBridgeMessageQueue.obj
 0001:000011cc       ??1AccessBridgeQueueElement@@QEAA@XZ 00000001800021cc f   AccessBridgeMessageQueue.obj
 0001:000011d8       ??1bad_alloc@std@@UEAA@XZ  00000001800021d8 f i AccessBridgeMessageQueue.obj
 0001:000011d8       ??1bad_array_new_length@std@@UEAA@XZ 00000001800021d8 f i MSVCRT:throw_bad_alloc.obj
 0001:000011ec       ??_Ebad_alloc@std@@UEAAPEAXI@Z 00000001800021ec f i AccessBridgeMessageQueue.obj
 0001:000011ec       ??_Ebad_array_new_length@std@@UEAAPEAXI@Z 00000001800021ec f i MSVCRT:throw_bad_alloc.obj
 0001:000011ec       ??_Eexception@std@@UEAAPEAXI@Z 00000001800021ec f i AccessBridgeMessageQueue.obj
 0001:000011ec       ??_Gbad_alloc@std@@UEAAPEAXI@Z 00000001800021ec f i AccessBridgeMessageQueue.obj
 0001:000011ec       ??_Gbad_array_new_length@std@@UEAAPEAXI@Z 00000001800021ec f i MSVCRT:throw_bad_alloc.obj
 0001:000011ec       ??_Gexception@std@@UEAAPEAXI@Z 00000001800021ec f i AccessBridgeMessageQueue.obj
 0001:00001230       ?add@AccessBridgeMessageQueue@@QEAA?AW4QueueReturns@@PEAVAccessBridgeQueueElement@@@Z 0000000180002230 f   AccessBridgeMessageQueue.obj
 0001:000012f4       ?getEventsWaiting@AccessBridgeMessageQueue@@QEAAHXZ 00000001800022f4 f   AccessBridgeMessageQueue.obj
 0001:000012f8       ?getRemoveLockSetting@AccessBridgeMessageQueue@@QEAAHXZ 00000001800022f8 f   AccessBridgeMessageQueue.obj
 0001:000012fc       ?remove@AccessBridgeMessageQueue@@QEAA?AW4QueueReturns@@PEAPEAVAccessBridgeQueueElement@@@Z 00000001800022fc f   AccessBridgeMessageQueue.obj
 0001:000013c0       ?setRemoveLock@AccessBridgeMessageQueue@@QEAA?AW4QueueReturns@@H@Z 00000001800023c0 f   AccessBridgeMessageQueue.obj
 0001:000013d4       ?what@exception@std@@UEBAPEBDXZ 00000001800023d4 f i AccessBridgeMessageQueue.obj
 0001:000013e8       ?initBroadcastMessageIDs@@YAHXZ 00000001800023e8 f   AccessBridgeMessages.obj
 0001:00001428       Windows_run                0000000180002428 f   AccessBridgeWindowsEntryPoints.obj
 0001:00001444       activateAccessibleHyperlink 0000000180002444 f   AccessBridgeWindowsEntryPoints.obj
 0001:00001464       addAccessibleSelectionFromContext 0000000180002464 f   AccessBridgeWindowsEntryPoints.obj
 0001:00001488       clearAccessibleSelectionFromContext 0000000180002488 f   AccessBridgeWindowsEntryPoints.obj
 0001:000014ac       doAccessibleActions        00000001800024ac f   AccessBridgeWindowsEntryPoints.obj
 0001:000014dc       getAccessibleActions       00000001800024dc f   AccessBridgeWindowsEntryPoints.obj
 0001:000014fc       getAccessibleChildFromContext 00000001800024fc f   AccessBridgeWindowsEntryPoints.obj
 0001:0000151c       getAccessibleContextAt     000000018000251c f   AccessBridgeWindowsEntryPoints.obj
 0001:00001558       getAccessibleContextFromHWND 0000000180002558 f   AccessBridgeWindowsEntryPoints.obj
 0001:00001578       getAccessibleContextInfo   0000000180002578 f   AccessBridgeWindowsEntryPoints.obj
 0001:00001598       getAccessibleContextWithFocus 0000000180002598 f   AccessBridgeWindowsEntryPoints.obj
 0001:000015b8       getAccessibleHyperlink     00000001800025b8 f   AccessBridgeWindowsEntryPoints.obj
 0001:000015e8       getAccessibleHyperlinkCount 00000001800025e8 f   AccessBridgeWindowsEntryPoints.obj
 0001:00001604       getAccessibleHypertext     0000000180002604 f   AccessBridgeWindowsEntryPoints.obj
 0001:00001624       getAccessibleHypertextExt  0000000180002624 f   AccessBridgeWindowsEntryPoints.obj
 0001:00001654       getAccessibleHypertextLinkIndex 0000000180002654 f   AccessBridgeWindowsEntryPoints.obj
 0001:00001674       getAccessibleIcons         0000000180002674 f   AccessBridgeWindowsEntryPoints.obj
 0001:00001694       getAccessibleKeyBindings   0000000180002694 f   AccessBridgeWindowsEntryPoints.obj
 0001:000016b4       getAccessibleParentFromContext 00000001800026b4 f   AccessBridgeWindowsEntryPoints.obj
 0001:000016d0       getAccessibleRelationSet   00000001800026d0 f   AccessBridgeWindowsEntryPoints.obj
 0001:000016f0       getAccessibleSelectionCountFromContext 00000001800026f0 f   AccessBridgeWindowsEntryPoints.obj
 0001:0000170c       getAccessibleSelectionFromContext 000000018000270c f   AccessBridgeWindowsEntryPoints.obj
 0001:0000172c       getAccessibleTableCellInfo 000000018000272c f   AccessBridgeWindowsEntryPoints.obj
 0001:00001768       getAccessibleTableColumn   0000000180002768 f   AccessBridgeWindowsEntryPoints.obj
 0001:00001788       getAccessibleTableColumnDescription 0000000180002788 f   AccessBridgeWindowsEntryPoints.obj
 0001:000017a8       getAccessibleTableColumnHeader 00000001800027a8 f   AccessBridgeWindowsEntryPoints.obj
 0001:000017c8       getAccessibleTableColumnSelectionCount 00000001800027c8 f   AccessBridgeWindowsEntryPoints.obj
 0001:000017e4       getAccessibleTableColumnSelections 00000001800027e4 f   AccessBridgeWindowsEntryPoints.obj
 0001:00001814       getAccessibleTableIndex    0000000180002814 f   AccessBridgeWindowsEntryPoints.obj
 0001:00001844       getAccessibleTableInfo     0000000180002844 f   AccessBridgeWindowsEntryPoints.obj
 0001:00001864       getAccessibleTableRow      0000000180002864 f   AccessBridgeWindowsEntryPoints.obj
 0001:00001884       getAccessibleTableRowDescription 0000000180002884 f   AccessBridgeWindowsEntryPoints.obj
 0001:000018a4       getAccessibleTableRowHeader 00000001800028a4 f   AccessBridgeWindowsEntryPoints.obj
 0001:000018c4       getAccessibleTableRowSelectionCount 00000001800028c4 f   AccessBridgeWindowsEntryPoints.obj
 0001:000018e0       getAccessibleTableRowSelections 00000001800028e0 f   AccessBridgeWindowsEntryPoints.obj
 0001:00001910       getAccessibleTextAttributes 0000000180002910 f   AccessBridgeWindowsEntryPoints.obj
 0001:00001940       getAccessibleTextInfo      0000000180002940 f   AccessBridgeWindowsEntryPoints.obj
 0001:00001978       getAccessibleTextItems     0000000180002978 f   AccessBridgeWindowsEntryPoints.obj
 0001:000019a8       getAccessibleTextLineBounds 00000001800029a8 f   AccessBridgeWindowsEntryPoints.obj
 0001:000019e4       getAccessibleTextRange     00000001800029e4 f   AccessBridgeWindowsEntryPoints.obj
 0001:00001a28       getAccessibleTextRect      0000000180002a28 f   AccessBridgeWindowsEntryPoints.obj
 0001:00001a58       getAccessibleTextSelectionInfo 0000000180002a58 f   AccessBridgeWindowsEntryPoints.obj
 0001:00001a78       getActiveDescendent        0000000180002a78 f   AccessBridgeWindowsEntryPoints.obj
 0001:00001a94       getCaretLocation           0000000180002a94 f   AccessBridgeWindowsEntryPoints.obj
 0001:00001ac4       getCurrentAccessibleValueFromContext 0000000180002ac4 f   AccessBridgeWindowsEntryPoints.obj
 0001:00001af4       getEventsWaiting           0000000180002af4 f   AccessBridgeWindowsEntryPoints.obj
 0001:00001b08       getHWNDFromAccessibleContext 0000000180002b08 f   AccessBridgeWindowsEntryPoints.obj
 0001:00001b24       getMaximumAccessibleValueFromContext 0000000180002b24 f   AccessBridgeWindowsEntryPoints.obj
 0001:00001b54       getMinimumAccessibleValueFromContext 0000000180002b54 f   AccessBridgeWindowsEntryPoints.obj
 0001:00001b84       getObjectDepth             0000000180002b84 f   AccessBridgeWindowsEntryPoints.obj
 0001:00001ba0       getParentWithRole          0000000180002ba0 f   AccessBridgeWindowsEntryPoints.obj
 0001:00001bc0       getParentWithRoleElseRoot  0000000180002bc0 f   AccessBridgeWindowsEntryPoints.obj
 0001:00001be0       getTextAttributesInRange   0000000180002be0 f   AccessBridgeWindowsEntryPoints.obj
 0001:00001c24       getTopLevelHWND            0000000180002c24 f   AccessBridgeWindowsEntryPoints.obj
 0001:00001c70       getTopLevelObject          0000000180002c70 f   AccessBridgeWindowsEntryPoints.obj
 0001:00001c8c       getVersionInfo             0000000180002c8c f   AccessBridgeWindowsEntryPoints.obj
 0001:00001cb0       getVirtualAccessibleName   0000000180002cb0 f   AccessBridgeWindowsEntryPoints.obj
 0001:00001ce0       getVisibleChildren         0000000180002ce0 f   AccessBridgeWindowsEntryPoints.obj
 0001:00001d10       getVisibleChildrenCount    0000000180002d10 f   AccessBridgeWindowsEntryPoints.obj
 0001:00001d2c       isAccessibleChildSelectedFromContext 0000000180002d2c f   AccessBridgeWindowsEntryPoints.obj
 0001:00001d4c       isAccessibleTableColumnSelected 0000000180002d4c f   AccessBridgeWindowsEntryPoints.obj
 0001:00001d6c       isAccessibleTableRowSelected 0000000180002d6c f   AccessBridgeWindowsEntryPoints.obj
 0001:00001d8c       isJavaWindow               0000000180002d8c f   AccessBridgeWindowsEntryPoints.obj
 0001:00001da4       isSameObject               0000000180002da4 f   AccessBridgeWindowsEntryPoints.obj
 0001:00001df4       releaseJavaObject          0000000180002df4 f   AccessBridgeWindowsEntryPoints.obj
 0001:00001e18       removeAccessibleSelectionFromContext 0000000180002e18 f   AccessBridgeWindowsEntryPoints.obj
 0001:00001e3c       requestFocus               0000000180002e3c f   AccessBridgeWindowsEntryPoints.obj
 0001:00001e58       selectAllAccessibleSelectionFromContext 0000000180002e58 f   AccessBridgeWindowsEntryPoints.obj
 0001:00001e7c       selectTextRange            0000000180002e7c f   AccessBridgeWindowsEntryPoints.obj
 0001:00001eac       setCaretPosition           0000000180002eac f   AccessBridgeWindowsEntryPoints.obj
 0001:00001ecc       setCaretUpdateFP           0000000180002ecc f   AccessBridgeWindowsEntryPoints.obj
 0001:00001eec       setFocusGainedFP           0000000180002eec f   AccessBridgeWindowsEntryPoints.obj
 0001:00001f0c       setFocusLostFP             0000000180002f0c f   AccessBridgeWindowsEntryPoints.obj
 0001:00001f2c       setJavaShutdownFP          0000000180002f2c f   AccessBridgeWindowsEntryPoints.obj
 0001:00001f4c       setMenuCanceledFP          0000000180002f4c f   AccessBridgeWindowsEntryPoints.obj
 0001:00001f6c       setMenuDeselectedFP        0000000180002f6c f   AccessBridgeWindowsEntryPoints.obj
 0001:00001f8c       setMenuSelectedFP          0000000180002f8c f   AccessBridgeWindowsEntryPoints.obj
 0001:00001fac       setMouseClickedFP          0000000180002fac f   AccessBridgeWindowsEntryPoints.obj
 0001:00001fcc       setMouseEnteredFP          0000000180002fcc f   AccessBridgeWindowsEntryPoints.obj
 0001:00001fec       setMouseExitedFP           0000000180002fec f   AccessBridgeWindowsEntryPoints.obj
 0001:0000200c       setMousePressedFP          000000018000300c f   AccessBridgeWindowsEntryPoints.obj
 0001:0000202c       setMouseReleasedFP         000000018000302c f   AccessBridgeWindowsEntryPoints.obj
 0001:0000204c       setPopupMenuCanceledFP     000000018000304c f   AccessBridgeWindowsEntryPoints.obj
 0001:0000206c       setPopupMenuWillBecomeInvisibleFP 000000018000306c f   AccessBridgeWindowsEntryPoints.obj
 0001:0000208c       setPopupMenuWillBecomeVisibleFP 000000018000308c f   AccessBridgeWindowsEntryPoints.obj
 0001:000020ac       setPropertyActiveDescendentChangeFP 00000001800030ac f   AccessBridgeWindowsEntryPoints.obj
 0001:000020cc       setPropertyCaretChangeFP   00000001800030cc f   AccessBridgeWindowsEntryPoints.obj
 0001:000020ec       setPropertyChangeFP        00000001800030ec f   AccessBridgeWindowsEntryPoints.obj
 0001:0000210c       setPropertyChildChangeFP   000000018000310c f   AccessBridgeWindowsEntryPoints.obj
 0001:0000212c       setPropertyDescriptionChangeFP 000000018000312c f   AccessBridgeWindowsEntryPoints.obj
 0001:0000214c       setPropertyNameChangeFP    000000018000314c f   AccessBridgeWindowsEntryPoints.obj
 0001:0000216c       setPropertySelectionChangeFP 000000018000316c f   AccessBridgeWindowsEntryPoints.obj
 0001:0000218c       setPropertyStateChangeFP   000000018000318c f   AccessBridgeWindowsEntryPoints.obj
 0001:000021ac       setPropertyTableModelChangeFP 00000001800031ac f   AccessBridgeWindowsEntryPoints.obj
 0001:000021cc       setPropertyTextChangeFP    00000001800031cc f   AccessBridgeWindowsEntryPoints.obj
 0001:000021ec       setPropertyValueChangeFP   00000001800031ec f   AccessBridgeWindowsEntryPoints.obj
 0001:0000220c       setPropertyVisibleDataChangeFP 000000018000320c f   AccessBridgeWindowsEntryPoints.obj
 0001:0000222c       setTextContents            000000018000322c f   AccessBridgeWindowsEntryPoints.obj
 0001:0000224c       ??0WinAccessBridge@@QEAA@PEAUHINSTANCE__@@@Z 000000018000324c f   WinAccessBridge.obj
 0001:000022dc       ??1WinAccessBridge@@QEAA@XZ 00000001800032dc f   WinAccessBridge.obj
 0001:000023c4       ?JavaVMDestroyed@WinAccessBridge@@QEAAXPEAUHWND__@@@Z 00000001800033c4 f   WinAccessBridge.obj
 0001:0000246c       ?activateAccessibleHyperlink@WinAccessBridge@@QEAAHJ_J0@Z 000000018000346c f   WinAccessBridge.obj
 0001:00002514       ?addAccessibilityEventNotification@WinAccessBridge@@QEAAX_J@Z 0000000180003514 f   WinAccessBridge.obj
 0001:000025b4       ?addAccessibleSelectionFromContext@WinAccessBridge@@QEAAXJ_JH@Z 00000001800035b4 f   WinAccessBridge.obj
 0001:00002620       ?addJavaEventNotification@WinAccessBridge@@QEAAX_J@Z 0000000180003620 f   WinAccessBridge.obj
 0001:000026c0       ?clearAccessibleSelectionFromContext@WinAccessBridge@@QEAAXJ_J@Z 00000001800036c0 f   WinAccessBridge.obj
 0001:00002728       ?doAccessibleActions@WinAccessBridge@@QEAAHJ_JPEAUAccessibleActionsToDoTag@@PEAH@Z 0000000180003728 f   WinAccessBridge.obj
 0001:00002814       ?getAccessibleActions@WinAccessBridge@@QEAAHJ_JPEAUAccessibleActionsTag@@@Z 0000000180003814 f   WinAccessBridge.obj
 0001:000028f0       ?getAccessibleChildFromContext@WinAccessBridge@@QEAA_JJ_JH@Z 00000001800038f0 f   WinAccessBridge.obj
 0001:0000297c       ?getAccessibleContextAt@WinAccessBridge@@QEAAHJ_JHHPEA_J@Z 000000018000397c f   WinAccessBridge.obj
 0001:00002a20       ?getAccessibleContextFromHWND@WinAccessBridge@@QEAAHPEAUHWND__@@PEAJPEA_J@Z 0000000180003a20 f   WinAccessBridge.obj
 0001:00002b24       ?getAccessibleContextInfo@WinAccessBridge@@QEAAHJ_JPEAUAccessibleContextInfoTag@@@Z 0000000180003b24 f   WinAccessBridge.obj
 0001:00002c1c       ?getAccessibleContextWithFocus@WinAccessBridge@@QEAAHPEAUHWND__@@PEAJPEA_J@Z 0000000180003c1c f   WinAccessBridge.obj
 0001:00002cc8       ?getAccessibleHyperlink@WinAccessBridge@@QEAAHJ_JHPEAUAccessibleHyperlinkInfoTag@@@Z 0000000180003cc8 f   WinAccessBridge.obj
 0001:00002da4       ?getAccessibleHyperlinkCount@WinAccessBridge@@QEAAHJ_J@Z 0000000180003da4 f   WinAccessBridge.obj
 0001:00002e5c       ?getAccessibleHypertext@WinAccessBridge@@QEAAHJ_JPEAUAccessibleHypertextInfoTag@@@Z 0000000180003e5c f   WinAccessBridge.obj
 0001:00002f38       ?getAccessibleHypertextExt@WinAccessBridge@@QEAAHJ_JHPEAUAccessibleHypertextInfoTag@@@Z 0000000180003f38 f   WinAccessBridge.obj
 0001:0000304c       ?getAccessibleHypertextLinkIndex@WinAccessBridge@@QEAAHJ_JH@Z 000000018000404c f   WinAccessBridge.obj
 0001:00003118       ?getAccessibleIcons@WinAccessBridge@@QEAAHJ_JPEAUAccessibleIconsTag@@@Z 0000000180004118 f   WinAccessBridge.obj
 0001:000031f4       ?getAccessibleKeyBindings@WinAccessBridge@@QEAAHJ_JPEAUAccessibleKeyBindingsTag@@@Z 00000001800041f4 f   WinAccessBridge.obj
 0001:000032fc       ?getAccessibleParentFromContext@WinAccessBridge@@QEAA_JJ_J@Z 00000001800042fc f   WinAccessBridge.obj
 0001:0000338c       ?getAccessibleRelationSet@WinAccessBridge@@QEAAHJ_JPEAUAccessibleRelationSetInfoTag@@@Z 000000018000438c f   WinAccessBridge.obj
 0001:00003464       ?getAccessibleSelectionCountFromContext@WinAccessBridge@@QEAAHJ_J@Z 0000000180004464 f   WinAccessBridge.obj
 0001:000034d8       ?getAccessibleSelectionFromContext@WinAccessBridge@@QEAA_JJ_JH@Z 00000001800044d8 f   WinAccessBridge.obj
 0001:00003550       ?getAccessibleTableCellInfo@WinAccessBridge@@QEAAHJ_JHHPEAUAccessibleTableCellInfoTag@@@Z 0000000180004550 f   WinAccessBridge.obj
 0001:00003654       ?getAccessibleTableColumn@WinAccessBridge@@QEAAHJ_JH@Z 0000000180004654 f   WinAccessBridge.obj
 0001:00003700       ?getAccessibleTableColumnDescription@WinAccessBridge@@QEAA_JJ_JH@Z 0000000180004700 f   WinAccessBridge.obj
 0001:000037ac       ?getAccessibleTableColumnHeader@WinAccessBridge@@QEAAHJ_JPEAUAccessibleTableInfoTag@@@Z 00000001800047ac f   WinAccessBridge.obj
 0001:00003868       ?getAccessibleTableColumnSelectionCount@WinAccessBridge@@QEAAHJ_J@Z 0000000180004868 f   WinAccessBridge.obj
 0001:0000390c       ?getAccessibleTableColumnSelections@WinAccessBridge@@QEAAHJ_JHPEAH@Z 000000018000490c f   WinAccessBridge.obj
 0001:000039e4       ?getAccessibleTableIndex@WinAccessBridge@@QEAAHJ_JHH@Z 00000001800049e4 f   WinAccessBridge.obj
 0001:00003aa4       ?getAccessibleTableInfo@WinAccessBridge@@QEAAHJ_JPEAUAccessibleTableInfoTag@@@Z 0000000180004aa4 f   WinAccessBridge.obj
 0001:00003b64       ?getAccessibleTableRow@WinAccessBridge@@QEAAHJ_JH@Z 0000000180004b64 f   WinAccessBridge.obj
 0001:00003c10       ?getAccessibleTableRowDescription@WinAccessBridge@@QEAA_JJ_JH@Z 0000000180004c10 f   WinAccessBridge.obj
 0001:00003cbc       ?getAccessibleTableRowHeader@WinAccessBridge@@QEAAHJ_JPEAUAccessibleTableInfoTag@@@Z 0000000180004cbc f   WinAccessBridge.obj
 0001:00003d78       ?getAccessibleTableRowSelectionCount@WinAccessBridge@@QEAAHJ_J@Z 0000000180004d78 f   WinAccessBridge.obj
 0001:00003e1c       ?getAccessibleTableRowSelections@WinAccessBridge@@QEAAHJ_JHPEAH@Z 0000000180004e1c f   WinAccessBridge.obj
 0001:00003ef4       ?getAccessibleTextAttributes@WinAccessBridge@@QEAAHJ_JHPEAUAccessibleTextAttributesInfoTag@@@Z 0000000180004ef4 f   WinAccessBridge.obj
 0001:00003fb0       ?getAccessibleTextInfo@WinAccessBridge@@QEAAHJ_JPEAUAccessibleTextInfoTag@@HH@Z 0000000180004fb0 f   WinAccessBridge.obj
 0001:0000408c       ?getAccessibleTextItems@WinAccessBridge@@QEAAHJ_JPEAUAccessibleTextItemsInfoTag@@H@Z 000000018000508c f   WinAccessBridge.obj
 0001:00004160       ?getAccessibleTextLineBounds@WinAccessBridge@@QEAAHJ_JHPEAH1@Z 0000000180005160 f   WinAccessBridge.obj
 0001:00004208       ?getAccessibleTextRange@WinAccessBridge@@QEAAHJ_JHHPEAGF@Z 0000000180005208 f   WinAccessBridge.obj
 0001:000042d8       ?getAccessibleTextRect@WinAccessBridge@@QEAAHJ_JPEAUAccessibleTextRectInfoTag@@H@Z 00000001800052d8 f   WinAccessBridge.obj
 0001:00004384       ?getAccessibleTextSelectionInfo@WinAccessBridge@@QEAAHJ_JPEAUAccessibleTextSelectionInfoTag@@@Z 0000000180005384 f   WinAccessBridge.obj
 0001:00004430       ?getActiveDescendent@WinAccessBridge@@QEAA_JJ_J@Z 0000000180005430 f   WinAccessBridge.obj
 0001:000044c0       ?getCaretLocation@WinAccessBridge@@QEAAHJ_JPEAUAccessibleTextRectInfoTag@@H@Z 00000001800054c0 f   WinAccessBridge.obj
 0001:0000456c       ?getCurrentAccessibleValueFromContext@WinAccessBridge@@QEAAHJ_JPEAGF@Z 000000018000556c f   WinAccessBridge.obj
 0001:00004614       ?getEventsWaiting@WinAccessBridge@@QEAAHXZ 0000000180005614 f   WinAccessBridge.obj
 0001:00004624       ?getHWNDFromAccessibleContext@WinAccessBridge@@QEAAPEAUHWND__@@J_J@Z 0000000180005624 f   WinAccessBridge.obj
 0001:000046bc       ?getMaximumAccessibleValueFromContext@WinAccessBridge@@QEAAHJ_JPEAGF@Z 00000001800056bc f   WinAccessBridge.obj
 0001:00004764       ?getMinimumAccessibleValueFromContext@WinAccessBridge@@QEAAHJ_JPEAGF@Z 0000000180005764 f   WinAccessBridge.obj
 0001:0000480c       ?getObjectDepth@WinAccessBridge@@QEAAHJ_J@Z 000000018000580c f   WinAccessBridge.obj
 0001:0000489c       ?getParentWithRole@WinAccessBridge@@QEAA_JJ_JPEBG@Z 000000018000589c f   WinAccessBridge.obj
 0001:00004984       ?getParentWithRoleElseRoot@WinAccessBridge@@QEAA_JJ_JPEBG@Z 0000000180005984 f   WinAccessBridge.obj
 0001:00004a38       ?getTextAttributesInRange@WinAccessBridge@@QEAAHJ_JHHPEAUAccessibleTextAttributesInfoTag@@PEAF@Z 0000000180005a38 f   WinAccessBridge.obj
 0001:00004b44       ?getTopLevelObject@WinAccessBridge@@QEAA_JJ_J@Z 0000000180005b44 f   WinAccessBridge.obj
 0001:00004bd4       ?getVersionInfo@WinAccessBridge@@QEAAHJPEAUAccessBridgeVersionInfoTag@@@Z 0000000180005bd4 f   WinAccessBridge.obj
 0001:00004ca8       ?getVirtualAccessibleName@WinAccessBridge@@QEAAHJ_JPEAGH@Z 0000000180005ca8 f   WinAccessBridge.obj
 0001:00004d84       ?getVisibleChildren@WinAccessBridge@@QEAAHJ_JHPEAUVisibleChildenInfoTag@@@Z 0000000180005d84 f   WinAccessBridge.obj
 0001:00004e3c       ?getVisibleChildrenCount@WinAccessBridge@@QEAAHJ_J@Z 0000000180005e3c f   WinAccessBridge.obj
 0001:00004ecc       ?initWindow@WinAccessBridge@@QEAAHXZ 0000000180005ecc f   WinAccessBridge.obj
 0001:00004f2c       ?isAccessibleChildSelectedFromContext@WinAccessBridge@@QEAAHJ_JH@Z 0000000180005f2c f   WinAccessBridge.obj
 0001:00004fb4       ?isAccessibleTableColumnSelected@WinAccessBridge@@QEAAHJ_JH@Z 0000000180005fb4 f   WinAccessBridge.obj
 0001:0000506c       ?isAccessibleTableRowSelected@WinAccessBridge@@QEAAHJ_JH@Z 000000018000606c f   WinAccessBridge.obj
 0001:00005124       ?isJavaWindow@WinAccessBridge@@QEAAHPEAUHWND__@@@Z 0000000180006124 f   WinAccessBridge.obj
 0001:000051ec       ?isSameObject@WinAccessBridge@@QEAAHJ_J0@Z 00000001800061ec f   WinAccessBridge.obj
 0001:000052b0       ?preProcessPackage@WinAccessBridge@@QEAAXPEADJ@Z 00000001800062b0 f   WinAccessBridge.obj
 0001:000053bc       ?processPackage@WinAccessBridge@@QEAAXPEADJ@Z 00000001800063bc f   WinAccessBridge.obj
 0001:00005b58       ?queuePackage@WinAccessBridge@@QEAAHPEADJ@Z 0000000180006b58 f   WinAccessBridge.obj
 0001:00005bcc       ?receiveAQueuedPackage@WinAccessBridge@@QEAAHXZ 0000000180006bcc f   WinAccessBridge.obj
 0001:00005d04       ?releaseJavaObject@WinAccessBridge@@QEAAXJ_J@Z 0000000180006d04 f   WinAccessBridge.obj
 0001:00005d80       ?removeAccessibilityEventNotification@WinAccessBridge@@QEAAX_J@Z 0000000180006d80 f   WinAccessBridge.obj
 0001:00005e20       ?removeAccessibleSelectionFromContext@WinAccessBridge@@QEAAXJ_JH@Z 0000000180006e20 f   WinAccessBridge.obj
 0001:00005e8c       ?removeJavaEventNotification@WinAccessBridge@@QEAAX_J@Z 0000000180006e8c f   WinAccessBridge.obj
 0001:00005f2c       ?rendezvousWithNewJavaDLL@WinAccessBridge@@QEAA_JPEAUHWND__@@J@Z 0000000180006f2c f   WinAccessBridge.obj
 0001:00006004       ?requestFocus@WinAccessBridge@@QEAAHJ_J@Z 0000000180007004 f   WinAccessBridge.obj
 0001:0000608c       ?selectAllAccessibleSelectionFromContext@WinAccessBridge@@QEAAXJ_J@Z 000000018000708c f   WinAccessBridge.obj
 0001:000060f4       ?selectTextRange@WinAccessBridge@@QEAAHJ_JHH@Z 00000001800070f4 f   WinAccessBridge.obj
 0001:00006190       ?sendMemoryPackage@WinAccessBridge@@QEAAHPEADJPEAUHWND__@@@Z 0000000180007190 f   WinAccessBridge.obj
 0001:000061f8       ?sendPackage@WinAccessBridge@@QEAAXPEADJPEAUHWND__@@@Z 00000001800071f8 f   WinAccessBridge.obj
 0001:0000622c       ?setCaretPosition@WinAccessBridge@@QEAAHJ_JH@Z 000000018000722c f   WinAccessBridge.obj
 0001:000062b8       ?setCaretUpdateFP@WinAccessBridge@@QEAAXP6AXJ_J0@Z@Z 00000001800072b8 f   WinAccessBridge.obj
 0001:000062c4       ?setFocusGainedFP@WinAccessBridge@@QEAAXP6AXJ_J0@Z@Z 00000001800072c4 f   WinAccessBridge.obj
 0001:000062d0       ?setFocusLostFP@WinAccessBridge@@QEAAXP6AXJ_J0@Z@Z 00000001800072d0 f   WinAccessBridge.obj
 0001:000062dc       ?setJavaShutdownFP@WinAccessBridge@@QEAAXP6AXJ@Z@Z 00000001800072dc f   WinAccessBridge.obj
 0001:000062e8       ?setMenuCanceledFP@WinAccessBridge@@QEAAXP6AXJ_J0@Z@Z 00000001800072e8 f   WinAccessBridge.obj
 0001:000062f4       ?setMenuDeselectedFP@WinAccessBridge@@QEAAXP6AXJ_J0@Z@Z 00000001800072f4 f   WinAccessBridge.obj
 0001:00006300       ?setMenuSelectedFP@WinAccessBridge@@QEAAXP6AXJ_J0@Z@Z 0000000180007300 f   WinAccessBridge.obj
 0001:0000630c       ?setMouseClickedFP@WinAccessBridge@@QEAAXP6AXJ_J0@Z@Z 000000018000730c f   WinAccessBridge.obj
 0001:00006318       ?setMouseEnteredFP@WinAccessBridge@@QEAAXP6AXJ_J0@Z@Z 0000000180007318 f   WinAccessBridge.obj
 0001:00006324       ?setMouseExitedFP@WinAccessBridge@@QEAAXP6AXJ_J0@Z@Z 0000000180007324 f   WinAccessBridge.obj
 0001:00006330       ?setMousePressedFP@WinAccessBridge@@QEAAXP6AXJ_J0@Z@Z 0000000180007330 f   WinAccessBridge.obj
 0001:0000633c       ?setMouseReleasedFP@WinAccessBridge@@QEAAXP6AXJ_J0@Z@Z 000000018000733c f   WinAccessBridge.obj
 0001:00006348       ?setPopupMenuCanceledFP@WinAccessBridge@@QEAAXP6AXJ_J0@Z@Z 0000000180007348 f   WinAccessBridge.obj
 0001:00006354       ?setPopupMenuWillBecomeInvisibleFP@WinAccessBridge@@QEAAXP6AXJ_J0@Z@Z 0000000180007354 f   WinAccessBridge.obj
 0001:00006360       ?setPopupMenuWillBecomeVisibleFP@WinAccessBridge@@QEAAXP6AXJ_J0@Z@Z 0000000180007360 f   WinAccessBridge.obj
 0001:0000636c       ?setPropertyActiveDescendentChangeFP@WinAccessBridge@@QEAAXP6AXJ_J000@Z@Z 000000018000736c f   WinAccessBridge.obj
 0001:00006378       ?setPropertyCaretChangeFP@WinAccessBridge@@QEAAXP6AXJ_J0HH@Z@Z 0000000180007378 f   WinAccessBridge.obj
 0001:00006384       ?setPropertyChangeFP@WinAccessBridge@@QEAAXP6AXJ_J0PEAG11@Z@Z 0000000180007384 f   WinAccessBridge.obj
 0001:00006390       ?setPropertyChildChangeFP@WinAccessBridge@@QEAAXP6AXJ_J000@Z@Z 0000000180007390 f   WinAccessBridge.obj
 0001:0000639c       ?setPropertyDescriptionChangeFP@WinAccessBridge@@QEAAXP6AXJ_J0PEAG1@Z@Z 000000018000739c f   WinAccessBridge.obj
 0001:000063a8       ?setPropertyNameChangeFP@WinAccessBridge@@QEAAXP6AXJ_J0PEAG1@Z@Z 00000001800073a8 f   WinAccessBridge.obj
 0001:000063b4       ?setPropertySelectionChangeFP@WinAccessBridge@@QEAAXP6AXJ_J0@Z@Z 00000001800073b4 f   WinAccessBridge.obj
 0001:000063c0       ?setPropertyStateChangeFP@WinAccessBridge@@QEAAXP6AXJ_J0PEAG1@Z@Z 00000001800073c0 f   WinAccessBridge.obj
 0001:000063cc       ?setPropertyTableModelChangeFP@WinAccessBridge@@QEAAXP6AXJ_J0PEAG1@Z@Z 00000001800073cc f   WinAccessBridge.obj
 0001:000063d8       ?setPropertyTextChangeFP@WinAccessBridge@@QEAAXP6AXJ_J0@Z@Z 00000001800073d8 f   WinAccessBridge.obj
 0001:000063e4       ?setPropertyValueChangeFP@WinAccessBridge@@QEAAXP6AXJ_J0PEAG1@Z@Z 00000001800073e4 f   WinAccessBridge.obj
 0001:000063f0       ?setPropertyVisibleDataChangeFP@WinAccessBridge@@QEAAXP6AXJ_J0@Z@Z 00000001800073f0 f   WinAccessBridge.obj
 0001:000063fc       ?setTextContents@WinAccessBridge@@QEAAHJ_JPEBG@Z 00000001800073fc f   WinAccessBridge.obj
 0001:000064b8       AccessBridgeDialogProc     00000001800074b8 f   WinAccessBridge.obj
 0001:000065f0       DllMain                    00000001800075f0 f   WinAccessBridge.obj
 0001:0000667c       ??_U@YAPEAX_K@Z            000000018000767c f   MSVCRT:new_array.obj
 0001:00006684       ??3@YAXPEAX_K@Z            0000000180007684 f   MSVCRT:delete_scalar_size.obj
 0001:00006684       ??_V@YAXPEAX@Z             0000000180007684 f   MSVCRT:delete_array.obj
 0001:0000668c       __GSHandlerCheck           000000018000768c f   MSVCRT:gshandler.obj
 0001:000066ac       __GSHandlerCheckCommon     00000001800076ac f   MSVCRT:gshandler.obj
 0001:00006720       __security_check_cookie    0000000180007720 f   MSVCRT:amdsecgs.obj
 0001:00006740       ??_Etype_info@@UEAAPEAXI@Z 0000000180007740 f i MSVCRT:std_type_info_static.obj
 0001:00006740       ??_Gtype_info@@UEAAPEAXI@Z 0000000180007740 f i MSVCRT:std_type_info_static.obj
 0001:0000676c       ??2@YAPEAX_K@Z             000000018000776c f   MSVCRT:new_scalar.obj
 0001:000067c0       __chkstk                   00000001800077c0 f   MSVCRT:chkstk.obj
 0001:000067c0       _alloca_probe              00000001800077c0 f   MSVCRT:chkstk.obj
 0001:00006b30       _DllMainCRTStartup         0000000180007b30 f   MSVCRT:dll_dllmain.obj
 0001:00006b70       ??3@YAXPEAX@Z              0000000180007b70 f   MSVCRT:delete_scalar.obj
 0001:00006b78       __raise_securityfailure    0000000180007b78 f   MSVCRT:gs_report.obj
 0001:00006bac       __report_gsfailure         0000000180007bac f   MSVCRT:gs_report.obj
 0001:00006cf4       ??0bad_array_new_length@std@@QEAA@AEBV01@@Z 0000000180007cf4 f i MSVCRT:throw_bad_alloc.obj
 0001:00006d30       ??0bad_array_new_length@std@@QEAA@XZ 0000000180007d30 f i MSVCRT:throw_bad_alloc.obj
 0001:00006d50       ?__scrt_throw_std_bad_alloc@@YAXXZ 0000000180007d50 f   MSVCRT:throw_bad_alloc.obj
 0001:00006d70       ?__scrt_throw_std_bad_array_new_length@@YAXXZ 0000000180007d70 f   MSVCRT:throw_bad_alloc.obj
 0001:00006d90       __security_init_cookie     0000000180007d90 f   MSVCRT:gs_support.obj
 0001:00006e3c       ?__scrt_initialize_type_info@@YAXXZ 0000000180007e3c f   MSVCRT:tncleanup.obj
 0001:00006e4c       ?__scrt_uninitialize_type_info@@YAXXZ 0000000180007e4c f   MSVCRT:tncleanup.obj
 0001:00006e58       __local_stdio_scanf_options 0000000180007e58 f i MSVCRT:default_local_stdio_options.obj
 0001:00006e60       __scrt_initialize_default_local_stdio_options 0000000180007e60 f   MSVCRT:default_local_stdio_options.obj
 0001:00006e7c       __scrt_acquire_startup_lock 0000000180007e7c f   MSVCRT:utility.obj
 0001:00006eb8       __scrt_dllmain_after_initialize_c 0000000180007eb8 f   MSVCRT:utility.obj
 0001:00006eec       __scrt_dllmain_before_initialize_c 0000000180007eec f   MSVCRT:utility.obj
 0001:00006f04       __scrt_dllmain_crt_thread_attach 0000000180007f04 f   MSVCRT:utility.obj
 0001:00006f2c       __scrt_dllmain_crt_thread_detach 0000000180007f2c f   MSVCRT:utility.obj
 0001:00006f44       __scrt_dllmain_exception_filter 0000000180007f44 f   MSVCRT:utility.obj
 0001:00006fa4       __scrt_dllmain_uninitialize_c 0000000180007fa4 f   MSVCRT:utility.obj
 0001:00006fd4       __scrt_dllmain_uninitialize_critical 0000000180007fd4 f   MSVCRT:utility.obj
 0001:00006fe8       __scrt_initialize_crt      0000000180007fe8 f   MSVCRT:utility.obj
 0001:00007034       __scrt_initialize_onexit_tables 0000000180008034 f   MSVCRT:utility.obj
 0001:000070c0       __scrt_is_nonwritable_in_current_image 00000001800080c0 f   MSVCRT:utility.obj
 0001:00007158       __scrt_release_startup_lock 0000000180008158 f   MSVCRT:utility.obj
 0001:0000717c       __scrt_uninitialize_crt    000000018000817c f   MSVCRT:utility.obj
 0001:000071a8       __scrt_get_dyn_tls_init_callback 00000001800081a8 f   MSVCRT:dyn_tls_init.obj
 0001:000071b0       __crt_debugger_hook        00000001800081b0 f   MSVCRT:utility_desktop.obj
 0001:000071b8       __scrt_fastfail            00000001800081b8 f   MSVCRT:utility_desktop.obj
 0001:00007304       _RTC_Initialize            0000000180008304 f   MSVCRT:initsect.obj
 0001:00007340       _RTC_Terminate             0000000180008340 f   MSVCRT:initsect.obj
 0001:0000737c       __isa_available_init       000000018000837c f   MSVCRT:cpu_disp.obj
 0001:00007528       _get_startup_argv_mode     0000000180008528 f   MSVCRT:argv_mode.obj
 0001:00007530       __scrt_is_ucrt_dll_in_use  0000000180008530 f   MSVCRT:ucrt_detection.obj
 0001:00007540       memcpy                     0000000180008540 f   vcruntime:VCRUNTIME140.dll
 0001:00007546       memset                     0000000180008546 f   vcruntime:VCRUNTIME140.dll
 0001:0000754c       __std_exception_copy       000000018000854c f   vcruntime:VCRUNTIME140.dll
 0001:00007552       __std_exception_destroy    0000000180008552 f   vcruntime:VCRUNTIME140.dll
 0001:00007558       _CxxThrowException         0000000180008558 f   vcruntime:VCRUNTIME140.dll
 0001:0000755e       __C_specific_handler       000000018000855e f   vcruntime:VCRUNTIME140.dll
 0001:00007564       __std_type_info_destroy_list 0000000180008564 f   vcruntime:VCRUNTIME140.dll
 0001:0000756a       strlen                     000000018000856a f   ucrt:api-ms-win-crt-string-l1-1-0.dll
 0001:00007570       strcmp                     0000000180008570 f   ucrt:api-ms-win-crt-string-l1-1-0.dll
 0001:00007576       strcpy                     0000000180008576 f   ucrt:api-ms-win-crt-string-l1-1-0.dll
 0001:0000757c       free                       000000018000857c f   ucrt:api-ms-win-crt-heap-l1-1-0.dll
 0001:00007582       malloc                     0000000180008582 f   ucrt:api-ms-win-crt-heap-l1-1-0.dll
 0001:00007588       _callnewh                  0000000180008588 f   ucrt:api-ms-win-crt-heap-l1-1-0.dll
 0001:0000758e       _initterm                  000000018000858e f   ucrt:api-ms-win-crt-runtime-l1-1-0.dll
 0001:00007594       _initterm_e                0000000180008594 f   ucrt:api-ms-win-crt-runtime-l1-1-0.dll
 0001:0000759a       _seh_filter_dll            000000018000859a f   ucrt:api-ms-win-crt-runtime-l1-1-0.dll
 0001:000075a0       _configure_narrow_argv     00000001800085a0 f   ucrt:api-ms-win-crt-runtime-l1-1-0.dll
 0001:000075a6       _initialize_narrow_environment 00000001800085a6 f   ucrt:api-ms-win-crt-runtime-l1-1-0.dll
 0001:000075ac       _initialize_onexit_table   00000001800085ac f   ucrt:api-ms-win-crt-runtime-l1-1-0.dll
 0001:000075b2       _execute_onexit_table      00000001800085b2 f   ucrt:api-ms-win-crt-runtime-l1-1-0.dll
 0001:000075b8       _cexit                     00000001800085b8 f   ucrt:api-ms-win-crt-runtime-l1-1-0.dll
 0001:000075c0       __acrt_initialize          00000001800085c0 f   MSVCRT:ucrt_stubs.obj
 0001:000075c0       __acrt_thread_attach       00000001800085c0 f   MSVCRT:ucrt_stubs.obj
 0001:000075c0       __acrt_thread_detach       00000001800085c0 f   MSVCRT:ucrt_stubs.obj
 0001:000075c0       __acrt_uninitialize        00000001800085c0 f   MSVCRT:ucrt_stubs.obj
 0001:000075c0       __acrt_uninitialize_critical 00000001800085c0 f   MSVCRT:ucrt_stubs.obj
 0001:000075c0       __scrt_stub_for_acrt_initialize 00000001800085c0 f   MSVCRT:ucrt_stubs.obj
 0001:000075c0       __scrt_stub_for_acrt_thread_attach 00000001800085c0 f   MSVCRT:ucrt_stubs.obj
 0001:000075c0       __scrt_stub_for_acrt_thread_detach 00000001800085c0 f   MSVCRT:ucrt_stubs.obj
 0001:000075c0       __scrt_stub_for_acrt_uninitialize 00000001800085c0 f   MSVCRT:ucrt_stubs.obj
 0001:000075c0       __scrt_stub_for_acrt_uninitialize_critical 00000001800085c0 f   MSVCRT:ucrt_stubs.obj
 0001:000075c0       __vcrt_initialize          00000001800085c0 f   MSVCRT:ucrt_stubs.obj
 0001:000075c0       __vcrt_thread_attach       00000001800085c0 f   MSVCRT:ucrt_stubs.obj
 0001:000075c0       __vcrt_thread_detach       00000001800085c0 f   MSVCRT:ucrt_stubs.obj
 0001:000075c0       __vcrt_uninitialize        00000001800085c0 f   MSVCRT:ucrt_stubs.obj
 0001:000075c0       __vcrt_uninitialize_critical 00000001800085c0 f   MSVCRT:ucrt_stubs.obj
 0001:000075c4       __scrt_stub_for_is_c_termination_complete 00000001800085c4 f   MSVCRT:ucrt_stubs.obj
 0001:000075c4       _is_c_termination_complete 00000001800085c4 f   MSVCRT:ucrt_stubs.obj
 0001:000075e0       _guard_dispatch_icall_nop  00000001800085e0 f   MSVCRT:guard_dispatch.obj
 0001:00007600       _guard_xfg_dispatch_icall_nop 0000000180008600 f   MSVCRT:guard_xfg_dispatch.obj
 0002:00000000       __imp_GetLastError         0000000180009000     kernel32:KERNEL32.dll
 0002:00000008       __imp_GetSystemTimeAsFileTime 0000000180009008     kernel32:KERNEL32.dll
 0002:00000010       __imp_CloseHandle          0000000180009010     kernel32:KERNEL32.dll
 0002:00000018       __imp_EnterCriticalSection 0000000180009018     kernel32:KERNEL32.dll
 0002:00000020       __imp_LeaveCriticalSection 0000000180009020     kernel32:KERNEL32.dll
 0002:00000028       __imp_MapViewOfFile        0000000180009028     kernel32:KERNEL32.dll
 0002:00000030       __imp_UnmapViewOfFile      0000000180009030     kernel32:KERNEL32.dll
 0002:00000038       __imp_CreateFileMappingA   0000000180009038     kernel32:KERNEL32.dll
 0002:00000040       __imp_InitializeCriticalSection 0000000180009040     kernel32:KERNEL32.dll
 0002:00000048       __imp_IsDebuggerPresent    0000000180009048     kernel32:KERNEL32.dll
 0002:00000050       __imp_InitializeSListHead  0000000180009050     kernel32:KERNEL32.dll
 0002:00000058       __imp_GetCurrentThreadId   0000000180009058     kernel32:KERNEL32.dll
 0002:00000060       __imp_GetCurrentProcessId  0000000180009060     kernel32:KERNEL32.dll
 0002:00000068       __imp_QueryPerformanceCounter 0000000180009068     kernel32:KERNEL32.dll
 0002:00000070       __imp_IsProcessorFeaturePresent 0000000180009070     kernel32:KERNEL32.dll
 0002:00000078       __imp_TerminateProcess     0000000180009078     kernel32:KERNEL32.dll
 0002:00000080       __imp_GetCurrentProcess    0000000180009080     kernel32:KERNEL32.dll
 0002:00000088       __imp_SetUnhandledExceptionFilter 0000000180009088     kernel32:KERNEL32.dll
 0002:00000090       __imp_UnhandledExceptionFilter 0000000180009090     kernel32:KERNEL32.dll
 0002:00000098       __imp_RtlVirtualUnwind     0000000180009098     kernel32:KERNEL32.dll
 0002:000000a0       __imp_RtlLookupFunctionEntry 00000001800090a0     kernel32:KERNEL32.dll
 0002:000000a8       __imp_RtlCaptureContext    00000001800090a8     kernel32:KERNEL32.dll
 0002:000000b0       \177KERNEL32_NULL_THUNK_DATA 00000001800090b0     kernel32:KERNEL32.dll
 0002:000000b8       __imp_CreateDialogParamA   00000001800090b8     user32:USER32.dll
 0002:000000c0       __imp_DestroyWindow        00000001800090c0     user32:USER32.dll
 0002:000000c8       __imp_PostMessageA         00000001800090c8     user32:USER32.dll
 0002:000000d0       __imp_SendMessageA         00000001800090d0     user32:USER32.dll
 0002:000000d8       __imp_GetParent            00000001800090d8     user32:USER32.dll
 0002:000000e0       __imp_GetWindowLongA       00000001800090e0     user32:USER32.dll
 0002:000000e8       __imp_ShowWindow           00000001800090e8     user32:USER32.dll
 0002:000000f0       __imp_SendMessageTimeoutA  00000001800090f0     user32:USER32.dll
 0002:000000f8       __imp_RegisterWindowMessageA 00000001800090f8     user32:USER32.dll
 0002:00000100       __imp_IsWindow             0000000180009100     user32:USER32.dll
 0002:00000108       \177USER32_NULL_THUNK_DATA 0000000180009108     user32:USER32.dll
 0002:00000110       __imp_memcpy               0000000180009110     vcruntime:VCRUNTIME140.dll
 0002:00000118       __imp_memset               0000000180009118     vcruntime:VCRUNTIME140.dll
 0002:00000120       __imp___std_type_info_destroy_list 0000000180009120     vcruntime:VCRUNTIME140.dll
 0002:00000128       __imp___C_specific_handler 0000000180009128     vcruntime:VCRUNTIME140.dll
 0002:00000130       __imp__CxxThrowException   0000000180009130     vcruntime:VCRUNTIME140.dll
 0002:00000138       __imp___std_exception_copy 0000000180009138     vcruntime:VCRUNTIME140.dll
 0002:00000140       __imp___std_exception_destroy 0000000180009140     vcruntime:VCRUNTIME140.dll
 0002:00000148       \177VCRUNTIME140_NULL_THUNK_DATA 0000000180009148     vcruntime:VCRUNTIME140.dll
 0002:00000150       __imp_getenv               0000000180009150     ucrt:api-ms-win-crt-environment-l1-1-0.dll
 0002:00000158       \177api-ms-win-crt-environment-l1-1-0_NULL_THUNK_DATA 0000000180009158     ucrt:api-ms-win-crt-environment-l1-1-0.dll
 0002:00000160       __imp_malloc               0000000180009160     ucrt:api-ms-win-crt-heap-l1-1-0.dll
 0002:00000168       __imp_free                 0000000180009168     ucrt:api-ms-win-crt-heap-l1-1-0.dll
 0002:00000170       __imp__callnewh            0000000180009170     ucrt:api-ms-win-crt-heap-l1-1-0.dll
 0002:00000178       \177api-ms-win-crt-heap-l1-1-0_NULL_THUNK_DATA 0000000180009178     ucrt:api-ms-win-crt-heap-l1-1-0.dll
 0002:00000180       __imp__initialize_onexit_table 0000000180009180     ucrt:api-ms-win-crt-runtime-l1-1-0.dll
 0002:00000188       __imp__initialize_narrow_environment 0000000180009188     ucrt:api-ms-win-crt-runtime-l1-1-0.dll
 0002:00000190       __imp__cexit               0000000180009190     ucrt:api-ms-win-crt-runtime-l1-1-0.dll
 0002:00000198       __imp__configure_narrow_argv 0000000180009198     ucrt:api-ms-win-crt-runtime-l1-1-0.dll
 0002:000001a0       __imp__initterm_e          00000001800091a0     ucrt:api-ms-win-crt-runtime-l1-1-0.dll
 0002:000001a8       __imp__initterm            00000001800091a8     ucrt:api-ms-win-crt-runtime-l1-1-0.dll
 0002:000001b0       __imp__execute_onexit_table 00000001800091b0     ucrt:api-ms-win-crt-runtime-l1-1-0.dll
 0002:000001b8       __imp__seh_filter_dll      00000001800091b8     ucrt:api-ms-win-crt-runtime-l1-1-0.dll
 0002:000001c0       \177api-ms-win-crt-runtime-l1-1-0_NULL_THUNK_DATA 00000001800091c0     ucrt:api-ms-win-crt-runtime-l1-1-0.dll
 0002:000001c8       __imp___acrt_iob_func      00000001800091c8     ucrt:api-ms-win-crt-stdio-l1-1-0.dll
 0002:000001d0       __imp_fopen                00000001800091d0     ucrt:api-ms-win-crt-stdio-l1-1-0.dll
 0002:000001d8       __imp___stdio_common_vsprintf 00000001800091d8     ucrt:api-ms-win-crt-stdio-l1-1-0.dll
 0002:000001e0       __imp___stdio_common_vfprintf 00000001800091e0     ucrt:api-ms-win-crt-stdio-l1-1-0.dll
 0002:000001e8       __imp_fclose               00000001800091e8     ucrt:api-ms-win-crt-stdio-l1-1-0.dll
 0002:000001f0       \177api-ms-win-crt-stdio-l1-1-0_NULL_THUNK_DATA 00000001800091f0     ucrt:api-ms-win-crt-stdio-l1-1-0.dll
 0002:000001f8       __imp_strcmp               00000001800091f8     ucrt:api-ms-win-crt-string-l1-1-0.dll
 0002:00000200       __imp_strcpy               0000000180009200     ucrt:api-ms-win-crt-string-l1-1-0.dll
 0002:00000208       __imp_strncpy              0000000180009208     ucrt:api-ms-win-crt-string-l1-1-0.dll
 0002:00000210       __imp_strlen               0000000180009210     ucrt:api-ms-win-crt-string-l1-1-0.dll
 0002:00000218       __imp_wcsncpy              0000000180009218     ucrt:api-ms-win-crt-string-l1-1-0.dll
 0002:00000220       \177api-ms-win-crt-string-l1-1-0_NULL_THUNK_DATA 0000000180009220     ucrt:api-ms-win-crt-string-l1-1-0.dll
 0002:00000228       __guard_check_icall_fptr   0000000180009228     MSVCRT:guard_support.obj
 0002:00000230       __guard_xfg_check_icall_fptr 0000000180009230     MSVCRT:guard_support.obj
 0002:00000238       __guard_dispatch_icall_fptr 0000000180009238     MSVCRT:guard_support.obj
 0002:00000240       __guard_xfg_dispatch_icall_fptr 0000000180009240     MSVCRT:guard_support.obj
 0002:00000248       __guard_xfg_table_dispatch_icall_fptr 0000000180009248     MSVCRT:guard_support.obj
 0002:00000250       __castguard_check_failure_os_handled_fptr 0000000180009250     MSVCRT:guard_support.obj
 0002:00000258       __guard_memcpy_fptr        0000000180009258     vcruntime:softmemtag.obj
 0002:00000260       __xc_a                     0000000180009260     MSVCRT:initializers.obj
 0002:00000268       __xc_z                     0000000180009268     MSVCRT:initializers.obj
 0002:00000270       __xi_a                     0000000180009270     MSVCRT:initializers.obj
 0002:00000278       __xi_z                     0000000180009278     MSVCRT:initializers.obj
 0002:00000280       __xp_a                     0000000180009280     MSVCRT:initializers.obj
 0002:00000288       __xp_z                     0000000180009288     MSVCRT:initializers.obj
 0002:00000290       __xt_a                     0000000180009290     MSVCRT:initializers.obj
 0002:00000298       __xt_z                     0000000180009298     MSVCRT:initializers.obj
 0002:000002a0       ??_C@_0BJ@FKCDJFDK@JAVA_ACCESSBRIDGE_LOGDIR@ 00000001800092a0     AccessBridgeDebug.obj
 0002:000002bc       ??_C@_04FPOLKAEB@?4log@    00000001800092bc     AccessBridgeDebug.obj
 0002:000002c4       ??_C@_01NOFIACDB@w@        00000001800092c4     AccessBridgeDebug.obj
 0002:000002c8       ??_C@_04EINJHBMM@?6?$CFs?6@ 00000001800092c8     AccessBridgeDebug.obj
 0002:000002d0       ??_C@_0BH@PPBGFLKL@Could?5not?5open?5file?5?$CFs@ 00000001800092d0     AccessBridgeDebug.obj
 0002:000002e8       ??_C@_07IBOBEFLP@?$FL?$CFllu?$FN?5@ 00000001800092e8     AccessBridgeDebug.obj
 0002:000002f0       ??_C@_02PCIJFNDE@?$AN?6@   00000001800092f0     AccessBridgeDebug.obj
 0002:000002f8       ??_C@_0BH@BLGOOJIK@AccessBridge?9?$CFp?9?$CFp?4mmf@ 00000001800092f8     AccessBridgeJavaVMInstance.obj
 0002:00000310       ??_C@_03DJNNCAJF@OK?$DP@   0000000180009310     AccessBridgeJavaVMInstance.obj
 0002:00000314       ??_C@_03ONJMBPEK@OK?$CB@   0000000180009314     AccessBridgeJavaVMInstance.obj
 0002:00000318       ??_C@_0CP@JIGBIHFH@?$FLINFO?$FN?3?5In?5AccessBridgeVMInstan@ 0000000180009318     AccessBridgeJavaVMInstance.obj
 0002:00000348       ??_C@_0CH@KAGNBCII@?$FLINFO?$FN?3?5?5?5?5?5javaAccessBridgeWin@ 0000000180009348     AccessBridgeJavaVMInstance.obj
 0002:00000370       ??_C@_0CC@NKGMANMJ@?$FLINFO?$FN?3?5In?5findAccessBridgeWind@ 0000000180009370     AccessBridgeJavaVMInstance.obj
 0002:00000398       ??_C@_0CK@NBPNOPCH@?$FLINFO?$FN?3?5In?5findABJavaInstanceFr@ 0000000180009398     AccessBridgeJavaVMInstance.obj
 0002:000003d0       ??_7exception@std@@6B@     00000001800093d0     AccessBridgeMessageQueue.obj
 0002:000003e0       ??_C@_0BC@EOODALEL@Unknown?5exception@ 00000001800093e0     AccessBridgeMessageQueue.obj
 0002:00000400       ??_7bad_alloc@std@@6B@     0000000180009400     AccessBridgeMessageQueue.obj
 0002:00000410       ??_C@_0P@GHFPNOJB@bad?5allocation@ 0000000180009410     AccessBridgeMessageQueue.obj
 0002:00000420       ??_C@_0CN@EPCNBBKD@?$FLINFO?$FN?3?5?5?5in?5AccessBridgeMessag@ 0000000180009420     AccessBridgeMessageQueue.obj
 0002:00000450       ??_C@_0BM@FHOEMINC@?$FLINFO?$FN?3?5?5?5?5?5queue?5size?5?$DN?5?$CFd@ 0000000180009450     AccessBridgeMessageQueue.obj
 0002:00000470       ??_C@_0DF@PKPPNDEN@?$FLWARN?$FN?3?5?5?5?5?5queue?5was?5locked?$DL?5r@ 0000000180009470     AccessBridgeMessageQueue.obj
 0002:000004a8       ??_C@_0CF@CAPEOLCL@?$FLINFO?$FN?3?5?5?5?5?5adding?5element?5to?5q@ 00000001800094a8     AccessBridgeMessageQueue.obj
 0002:000004d0       ??_C@_0DL@IILCMNMG@?$FLINFO?$FN?3?5?5?5?5?5returning?5from?5Acce@ 00000001800094d0     AccessBridgeMessageQueue.obj
 0002:00000510       ??_C@_0DA@NHLJEKKG@?$FLINFO?$FN?3?5?5?5in?5AccessBridgeMessag@ 0000000180009510     AccessBridgeMessageQueue.obj
 0002:00000540       ??_C@_0CJ@FBOCEMKO@?$FLINFO?$FN?3?5?5?5?5?5removing?5element?5fr@ 0000000180009540     AccessBridgeMessageQueue.obj
 0002:00000570       ??_C@_0DO@NEJIEHGM@?$FLINFO?$FN?3?5?5?5?5?5returning?5from?5Acce@ 0000000180009570     AccessBridgeMessageQueue.obj
 0002:000005b0       ??_C@_0BM@BIAOFPJG@AccessBridge?9FromJava?9Hello@ 00000001800095b0     AccessBridgeMessages.obj
 0002:000005d0       ??_C@_0BP@OELHMMDF@AccessBridge?9FromWindows?9Hello@ 00000001800095d0     AccessBridgeMessages.obj
 0002:000005f0       ??_C@_0EC@DLPGLEGA@?$AN?6AccessBridgeWindowsEntryPoint@ 00000001800095f0     AccessBridgeWindowsEntryPoints.obj
 0002:00000638       ??_C@_0BG@GGFIABLO@windows_access_bridge@ 0000000180009638     WinAccessBridge.obj
 0002:00000650       ??_C@_0BL@GLCNGDJJ@?$FLINFO?$FN?3?5DLL_PROCESS_ATTACH@ 0000000180009650     WinAccessBridge.obj
 0002:00000670       ??_C@_0EG@HHOMJPNP@?$FLINFO?$FN?3?5?$CK?$CK?$CK?5AccessBridgeDialogP@ 0000000180009670     WinAccessBridge.obj
 0002:000006b8       ??_C@_0CP@LHINEKAP@?$FLINFO?$FN?3?5AccessBridgeDialogProc?5@ 00000001800096b8     WinAccessBridge.obj
 0002:000006f0       ??_C@_0EH@MDELPMEJ@?$FLINFO?$FN?3?5AccessBridgeDialogProc?5@ 00000001800096f0     WinAccessBridge.obj
 0002:00000738       ??_C@_0DP@HBEMDAPF@?$FLINFO?$FN?3?5AccessBridgeDialogProc?5@ 0000000180009738     WinAccessBridge.obj
 0002:00000780       ??_C@_0EH@MPLEACPJ@?$FLINFO?$FN?3?5AccessBridgeDialogProc?5@ 0000000180009780     WinAccessBridge.obj
 0002:000007d0       ??_C@_0EG@GGGHDKAD@?$FLINFO?$FN?3?5?$CK?$CK?$CK?$CK?$CK?5AccessBridgeDialo@ 00000001800097d0     WinAccessBridge.obj
 0002:00000818       ??_C@_0DE@BGNNIIOB@?$FLINFO?$FN?3?5?5?5javaVMs?5chain?5in?5use?0@ 0000000180009818     WinAccessBridge.obj
 0002:00000850       ??_C@_0CC@NEJJLLGC@?$FLINFO?$FN?3?5?5?5calling?5javaVMDestroy@ 0000000180009850     WinAccessBridge.obj
 0002:00000880       ??_C@_0FG@BHPCMIAO@?$FLINFO?$FN?3?5AccessBridgeDialogProc?5@ 0000000180009880     WinAccessBridge.obj
 0002:000008d8       ??_C@_0BN@FIPGEIKI@?$FLINFO?$FN?3?5WinAccessBridge?5ctor@ 00000001800098d8     WinAccessBridge.obj
 0002:000008f8       ??_C@_0DE@JFKNENGC@?$FLINFO?$FN?3?5?$CK?$CK?$CK?$CK?$CKin?5WinAccessBridge@ 00000001800098f8     WinAccessBridge.obj
 0002:00000930       ??_C@_0CG@EDMKMONP@?$FLINFO?$FN?3?5?5?5telling?5?$CFp?5we?8re?5goin@ 0000000180009930     WinAccessBridge.obj
 0002:00000958       ??_C@_0DB@CFPLAPDG@?$FLINFO?$FN?3?5?5?5finished?5telling?5JVMs@ 0000000180009958     WinAccessBridge.obj
 0002:00000990       ??_C@_0EE@GBJFCFOA@?$FLINFO?$FN?3?5?5?5finished?5deleting?5eve@ 0000000180009990     WinAccessBridge.obj
 0002:000009d8       ??_C@_0BP@EBFMIPOK@?$FLINFO?$FN?3?5GOODBYE?5CRUEL?5WORLD?4?4?4@ 00000001800099d8     WinAccessBridge.obj
 0002:000009f8       ??_C@_0BJ@LMONFDOG@ACCESSBRIDGESTATUSWINDOW@ 00000001800099f8     WinAccessBridge.obj
 0002:00000a18       ??_C@_0DN@NNELAOKC@?$FLINFO?$FN?3?5in?5WinAccessBridge?3?3ren@ 0000000180009a18     WinAccessBridge.obj
 0002:00000a58       ??_C@_0CJ@LMLGKPGD@?$FLINFO?$FN?3?5?5?5Setting?5Java?5event?5ma@ 0000000180009a58     WinAccessBridge.obj
 0002:00000a88       ??_C@_0DC@IJKHOBEO@?$FLINFO?$FN?3?5?5?5Setting?5Accessibility@ 0000000180009a88     WinAccessBridge.obj
 0002:00000ac0       ??_C@_0DN@ECLBFGAO@?$FLERROR?$FN?3?5Failed?5to?5initiate?5IPC@ 0000000180009ac0     WinAccessBridge.obj
 0002:00000b00       ??_C@_0DG@OEMNKFJP@?$FLINFO?$FN?3?5?5?5Success?$CB?$CB?5?5We?5rendezv@ 0000000180009b00     WinAccessBridge.obj
 0002:00000b38       ??_C@_0DK@BLMJEFJH@?$FLERROR?$FN?3?5sending?5memory?5package@ 0000000180009b38     WinAccessBridge.obj
 0002:00000b78       ??_C@_0DC@BABNPCOM@?$FLINFO?$FN?3?5?5in?5WinAccessBridge?3?3qu@ 0000000180009b78     WinAccessBridge.obj
 0002:00000bb0       ??_C@_0DE@NOAFOCML@?$FLINFO?$FN?3?5in?5WinAccessBridge?3?3rec@ 0000000180009bb0     WinAccessBridge.obj
 0002:00000be8       ??_C@_0BM@KNOOFOHJ@?$FLINFO?$FN?3?5?5dequeueing?5message@ 0000000180009be8     WinAccessBridge.obj
 0002:00000c08       ??_C@_0CD@GBHFIMOB@?$FLERROR?$FN?3?5Queue?5seems?5to?5be?5brok@ 0000000180009c08     WinAccessBridge.obj
 0002:00000c30       ??_C@_0CA@LFELFFDM@?$FLINFO?$FN?3?5?5found?5one?$DL?5sending?5it?$CB@ 0000000180009c30     WinAccessBridge.obj
 0002:00000c50       ??_C@_0BP@ENBFDBDP@?$FLWARN?$FN?3?5?5?5ODD?4?4?4?5element?5?$DN?$DN?50?$CB@ 0000000180009c50     WinAccessBridge.obj
 0002:00000c70       ??_C@_0CP@OIAJKCPF@?$FLWARN?$FN?3?5?5Queue?5in?5use?0?5will?5try@ 0000000180009c70     WinAccessBridge.obj
 0002:00000ca0       ??_C@_0DH@KAJCMPPF@?$FLWARN?$FN?3?5?5unable?5to?5dequeue?5mess@ 0000000180009ca0     WinAccessBridge.obj
 0002:00000cd8       ??_C@_0CO@KCIANNAF@?$FLINFO?$FN?3?5PreProcessing?5package?5s@ 0000000180009cd8     WinAccessBridge.obj
 0002:00000d10       ??_C@_0EF@DFMGOCJF@?$FLERROR?$FN?3?5?5?5processing?5FAILED?$CB?$CB?5@ 0000000180009d10     WinAccessBridge.obj
 0002:00000d58       ??_C@_0CL@HBCKEPEE@?$FLINFO?$FN?3?5?5?5?5package?5preprocessin@ 0000000180009d58     WinAccessBridge.obj
 0002:00000d88       ??_C@_0DM@CCADHAH@?$FLINFO?$FN?3?5WinAccessBridge?3?3Proces@ 0000000180009d88     WinAccessBridge.obj
 0002:00000dc8       ??_C@_0CI@KAACKIJC@?$FLINFO?$FN?3?5?5?5?5type?5?$DN?$DN?5cJavaShutdow@ 0000000180009dc8     WinAccessBridge.obj
 0002:00000df0       ??_C@_0CE@KGDIDFJM@?$FLINFO?$FN?3?5?5?5?5event?5callback?5compl@ 0000000180009df0     WinAccessBridge.obj
 0002:00000e18       ??_C@_0BI@MGOIGNJM@?$FLINFO?$FN?3?5?5?5?5event?5fired?$CB@ 0000000180009e18     WinAccessBridge.obj
 0002:00000e30       ??_C@_0EC@JELBKKLB@?$FLERROR?$FN?3?5?5?5?5processing?5FAILED?$CB?$CB@ 0000000180009e30     WinAccessBridge.obj
 0002:00000e78       ??_C@_0CM@OIHFPHBP@?$FLINFO?$FN?3?5?5?5?5begin?5callback?5to?5AT@ 0000000180009e78     WinAccessBridge.obj
 0002:00000eb0       ??_C@_0EB@PCOLNIOI@?$FLERROR?$FN?3?5?5?5processing?5FAILED?$CB?$CB?5@ 0000000180009eb0     WinAccessBridge.obj
 0002:00000f00       ??_C@_0EG@DADDGPDA@?$FLERROR?$FN?3?5?5?5?5processing?5FAILED?$CB?$CB@ 0000000180009f00     WinAccessBridge.obj
 0002:00000f48       ??_C@_0CI@PMGDCMNI@?$FLINFO?$FN?3?5?5?5?5package?5processing?5c@ 0000000180009f48     WinAccessBridge.obj
 0002:00000f70       ??_C@_0DD@EDMANGOO@?$FLINFO?$FN?3?5?$CK?$CK?$CK?$CK?$CK?5WinAccessBridge?3?3@ 0000000180009f70     WinAccessBridge.obj
 0002:00000fa8       ??_C@_0CP@IIHJFGGB@?$FLINFO?$FN?3?5?5?5data?5structures?5succe@ 0000000180009fa8     WinAccessBridge.obj
 0002:00000fd8       ??_C@_0DB@JABMCGEJ@?$FLERROR?$FN?3?5couldn?8t?5find?5matching@ 0000000180009fd8     WinAccessBridge.obj
 0002:00001010       ??_C@_0DJ@EFGAHBMH@?$FLINFO?$FN?3?5WinAccessBridge?3?3releas@ 000000018000a010     WinAccessBridge.obj
 0002:00001050       ??_C@_0CO@GDCOMIDN@?$FLINFO?$FN?3?5WinAccessBridge?3?3getVer@ 000000018000a050     WinAccessBridge.obj
 0002:00001080       ??_C@_0IH@JNMBAFNI@?$FLINFO?$FN?3?5?5?5VMversion?3?5?$CFls?6?5?5?5?5?5?5@ 000000018000a080     WinAccessBridge.obj
 0002:00001108       ??_C@_0CJ@MFBANPLF@?$FLINFO?$FN?3?5In?5WinAccessBridge?3?3isJ@ 000000018000a108     WinAccessBridge.obj
 0002:00001138       ??_C@_0CK@OIADIKJK@?$FLINFO?$FN?3?5WinAccessBridge?3?3isJava@ 000000018000a138     WinAccessBridge.obj
 0002:00001168       ??_C@_0DJ@GDIICFAI@?$FLINFO?$FN?3?5WinAccessBridge?3?3isSame@ 000000018000a168     WinAccessBridge.obj
 0002:000011b0       ??_C@_0EF@JHJAECO@?$FLINFO?$FN?3?5?5?5WinAccessBridge?3?3isSa@ 000000018000a1b0     WinAccessBridge.obj
 0002:00001200       ??_C@_0EL@EGCPHNBB@?$FLINFO?$FN?3?5?5?5WinAccessBridge?3?3isSa@ 000000018000a200     WinAccessBridge.obj
 0002:00001250       ??_C@_0FE@JNIGOBOL@?$FLERROR?$FN?3?5?5?5WinAccessBridge?3?3isS@ 000000018000a250     WinAccessBridge.obj
 0002:000012a8       ??_C@_0DM@KHCMPGEG@?$FLINFO?$FN?3?5WinAccessBridge?3?3getAcc@ 000000018000a2a8     WinAccessBridge.obj
 0002:000012e8       ??_C@_0DA@KDJKNLAN@?$FLINFO?$FN?3?5?5?5?5?5current?9?$DOvmID?5?$DN?5?$CFX?0@ 000000018000a2e8     WinAccessBridge.obj
 0002:00001318       ??_C@_0CP@IJNFIHAG@?$FLINFO?$FN?3?5?5?5?5?5pkg?9?$DOrAccessibleCon@ 000000018000a318     WinAccessBridge.obj
 0002:00001348       ??_C@_0DJ@FFBPMFOM@?$FLERROR?$FN?3?5getAccessibleContextFr@ 000000018000a348     WinAccessBridge.obj
 0002:00001388       ??_C@_0DO@IIGOCPCC@?$FLERROR?$FN?3?5getAccessibleContextFr@ 000000018000a388     WinAccessBridge.obj
 0002:000013c8       ??_C@_0DL@KEEIEGBJ@?$FLINFO?$FN?3?5?5?5in?5WinAccessBridge?3?3g@ 000000018000a3c8     WinAccessBridge.obj
 0002:00001410       ??_C@_0EA@HDGDGEMM@?$FLINFO?$FN?3?5WinAccessBridge?3?3getHWN@ 000000018000a410     WinAccessBridge.obj
 0002:00001450       ??_C@_0EA@FHJPOEHJ@?$FLINFO?$FN?3?5WinAccessBridge?3?3getAcc@ 000000018000a450     WinAccessBridge.obj
 0002:00001490       ??_C@_0EB@HKEAOAKG@?$FLINFO?$FN?3?5WinAccessBridge?3?3getAcc@ 000000018000a490     WinAccessBridge.obj
 0002:000014e0       ??_C@_0EC@OFBFCAEJ@?$FLINFO?$FN?3?5WinAccessBridge?3?3getAcc@ 000000018000a4e0     WinAccessBridge.obj
 0002:00001530       ??_C@_0JA@MODCAACP@?$FLINFO?$FN?3?5?5?5name?3?5?$CFls?6?5?5?5?5?5?5?5?5?5?5d@ 000000018000a530     WinAccessBridge.obj
 0002:000015c0       ??_C@_0EJ@HLHMECO@?$FLINFO?$FN?3?5WinAccessBridge?3?3getAcc@ 000000018000a5c0     WinAccessBridge.obj
 0002:00001610       ??_C@_0EA@MDGJLODH@?$FLINFO?$FN?3?5WinAccessBridge?3?3getAcc@ 000000018000a610     WinAccessBridge.obj
 0002:00001650       ??_C@_0EI@IEEMIFOJ@?$FLINFO?$FN?3?5?$CD?$CD?$CD?$CD?$CD?5WinAccessBridge?3?3@ 000000018000a650     WinAccessBridge.obj
 0002:000016a0       ??_C@_0EC@FNKONEFN@?$FLINFO?$FN?3?5?5?5?$CD?$CD?$CD?$CD?$CD?5WinAccessBridge@ 000000018000a6a0     WinAccessBridge.obj
 0002:000016f0       ??_C@_0EA@GPGOILHN@?$FLERROR?$FN?3?5?5?5?$CD?$CD?$CD?$CD?$CD?5WinAccessBridg@ 000000018000a6f0     WinAccessBridge.obj
 0002:00001730       ??_C@_0EO@GIFIOBJO@?$FLINFO?$FN?3?5?$CD?$CD?$CD?$CD?$CD?5WinAccessBridge?3?3@ 000000018000a730     WinAccessBridge.obj
 0002:00001780       ??_C@_0DK@FPHEFKPF@?$FLINFO?$FN?3?5?5?5XXXX?5pkg?9?$DOrTableCellI@ 000000018000a780     WinAccessBridge.obj
 0002:000017c0       ??_C@_0EG@CFNEHAJF@?$FLINFO?$FN?3?5?5?5?$CD?$CD?$CD?$CD?$CD?5WinAccessBridge@ 000000018000a7c0     WinAccessBridge.obj
 0002:00001810       ??_C@_0EE@DMEKGPAL@?$FLERROR?$FN?3?5?5?5?$CD?$CD?$CD?$CD?$CD?5WinAccessBridg@ 000000018000a810     WinAccessBridge.obj
 0002:00001860       ??_C@_0EJ@GHNOCBA@?$FLINFO?$FN?3?5?$CD?$CD?$CD?$CD?$CD?5WinAccessBridge?3?3@ 000000018000a860     WinAccessBridge.obj
 0002:000018b0       ??_C@_0EH@MMAIEADN@?$FLINFO?$FN?3?5?5?5?$CD?$CD?$CD?$CD?$CD?5WinAccessBridge@ 000000018000a8b0     WinAccessBridge.obj
 0002:00001900       ??_C@_0EF@IGPDOLOH@?$FLERROR?$FN?3?5?5?5?$CD?$CD?$CD?$CD?$CD?5WinAccessBridg@ 000000018000a900     WinAccessBridge.obj
 0002:00001950       ??_C@_0EM@KLDOANDG@?$FLINFO?$FN?3?5?$CD?$CD?$CD?$CD?$CD?5WinAccessBridge?3?3@ 000000018000a950     WinAccessBridge.obj
 0002:000019a0       ??_C@_0EK@DJMDCCLK@?$FLINFO?$FN?3?5?5?5?$CD?$CD?$CD?$CD?$CD?5WinAccessBridge@ 000000018000a9a0     WinAccessBridge.obj
 0002:000019f0       ??_C@_0EI@CELDDCKP@?$FLERROR?$FN?3?5?5?5?$CD?$CD?$CD?$CD?$CD?5WinAccessBridg@ 000000018000a9f0     WinAccessBridge.obj
 0002:00001a40       ??_C@_0FC@BPONCABC@?$FLINFO?$FN?3?5?$CD?$CD?$CD?$CD?$CD?5WinAccessBridge?3?3@ 000000018000aa40     WinAccessBridge.obj
 0002:00001aa0       ??_C@_0EM@JPIPIDPC@?$FLINFO?$FN?3?5?5?5?$CD?$CD?$CD?$CD?$CD?5WinAccessBridge@ 000000018000aaa0     WinAccessBridge.obj
 0002:00001af0       ??_C@_0EK@IGPCFPOI@?$FLERROR?$FN?3?5?5?5?$CD?$CD?$CD?$CD?$CD?5WinAccessBridg@ 000000018000aaf0     WinAccessBridge.obj
 0002:00001b40       ??_C@_0FF@GEJHIBCC@?$FLINFO?$FN?3?5?$CD?$CD?$CD?$CD?$CD?5WinAccessBridge?3?3@ 000000018000ab40     WinAccessBridge.obj
 0002:00001ba0       ??_C@_0EP@PJFHLMKB@?$FLINFO?$FN?3?5?5?5?$CD?$CD?$CD?$CD?$CD?5WinAccessBridge@ 000000018000aba0     WinAccessBridge.obj
 0002:00001bf0       ??_C@_0EN@FJIGOJNI@?$FLERROR?$FN?3?5?5?5?$CD?$CD?$CD?$CD?$CD?5WinAccessBridg@ 000000018000abf0     WinAccessBridge.obj
 0002:00001c40       ??_C@_0FB@IPIFJJKK@?$FLINFO?$FN?3?5?$CD?$CD?$CD?$CD?$CD?5WinAccessBridge?3?3@ 000000018000ac40     WinAccessBridge.obj
 0002:00001ca0       ??_C@_0EP@DHAGNOBO@?$FLINFO?$FN?3?5?5?5?$CD?$CD?$CD?$CD?$CD?5WinAccessBridge@ 000000018000aca0     WinAccessBridge.obj
 0002:00001cf0       ??_C@_0EN@IFAFODLF@?$FLERROR?$FN?3?5?5?5?$CD?$CD?$CD?$CD?$CD?5WinAccessBridg@ 000000018000acf0     WinAccessBridge.obj
 0002:00001d40       ??_C@_0EK@FCAMCNJB@?$FLINFO?$FN?3?5?$CD?$CD?$CD?$CD?$CD?5WinAccessBridge?3?3@ 000000018000ad40     WinAccessBridge.obj
 0002:00001d90       ??_C@_0EI@LCHMKLCB@?$FLINFO?$FN?3?5?5?5?$CD?$CD?$CD?$CD?$CD?5WinAccessBridge@ 000000018000ad90     WinAccessBridge.obj
 0002:00001de0       ??_C@_0EG@PCFFNJPM@?$FLERROR?$FN?3?5?5?5?$CD?$CD?$CD?$CD?$CD?5WinAccessBridg@ 000000018000ade0     WinAccessBridge.obj
 0002:00001e30       ??_C@_0EN@MHFLCDEG@?$FLINFO?$FN?3?5?$CD?$CD?$CD?$CD?$CD?5WinAccessBridge?3?3@ 000000018000ae30     WinAccessBridge.obj
 0002:00001e80       ??_C@_0EL@HPJEOBAF@?$FLINFO?$FN?3?5?5?5?$CD?$CD?$CD?$CD?$CD?5WinAccessBridge@ 000000018000ae80     WinAccessBridge.obj
 0002:00001ed0       ??_C@_0EJ@EFJNHGOC@?$FLERROR?$FN?3?5?5?5?$CD?$CD?$CD?$CD?$CD?5WinAccessBridg@ 000000018000aed0     WinAccessBridge.obj
 0002:00001f20       ??_C@_0FE@EEAPAHGA@?$FLINFO?$FN?3?5?$CD?$CD?$CD?$CD?$CD?5WinAccessBridge?3?3@ 000000018000af20     WinAccessBridge.obj
 0002:00001f80       ??_C@_0FC@IJCKDOEL@?$FLINFO?$FN?3?5?5?5?$CD?$CD?$CD?$CD?$CD?5WinAccessBridge@ 000000018000af80     WinAccessBridge.obj
 0002:00001fe0       ??_C@_0FA@EEJJLKOB@?$FLERROR?$FN?3?5?5?5?$CD?$CD?$CD?$CD?$CD?5WinAccessBridg@ 000000018000afe0     WinAccessBridge.obj
 0002:00002030       ??_C@_0EN@IKMAMDCJ@?$FLINFO?$FN?3?5?$CD?$CD?$CD?$CD?$CD?5WinAccessBridge?3?3@ 000000018000b030     WinAccessBridge.obj
 0002:00002080       ??_C@_0EL@MCFEFCEP@?$FLINFO?$FN?3?5?5?5?$CD?$CD?$CD?$CD?$CD?5WinAccessBridge@ 000000018000b080     WinAccessBridge.obj
 0002:000020d0       ??_C@_0EJ@OEGCIAEN@?$FLERROR?$FN?3?5?5?5?$CD?$CD?$CD?$CD?$CD?5WinAccessBridg@ 000000018000b0d0     WinAccessBridge.obj
 0002:00002120       ??_C@_0FB@FBDIFIGA@?$FLERROR?$FN?3?5?$CD?$CD?$CD?$CD?$CD?5WinAccessBridge?3@ 000000018000b120     WinAccessBridge.obj
 0002:00002180       ??_C@_0EO@KBJAHINP@?$FLINFO?$FN?3?5?5?5?$CD?$CD?$CD?$CD?$CD?5WinAccessBridge@ 000000018000b180     WinAccessBridge.obj
 0002:000021d0       ??_C@_0EM@FBMEIFEO@?$FLERROR?$FN?3?5?5?5?$CD?$CD?$CD?$CD?$CD?5WinAccessBridg@ 000000018000b1d0     WinAccessBridge.obj
 0002:00002220       ??_C@_0EN@EJPIGDNI@?$FLINFO?$FN?3?5?$CD?$CD?$CD?$CD?$CD?5WinAccessBridge?3?3@ 000000018000b220     WinAccessBridge.obj
 0002:00002270       ??_C@_0EB@EHNAMLGG@?$FLINFO?$FN?3?5?5?5?$CD?$CD?$CD?$CD?$CD?5WinAccessBridge@ 000000018000b270     WinAccessBridge.obj
 0002:000022b8       ??_C@_0DP@JGIKFGJD@?$FLERROR?$FN?3?5?5?5?$CD?$CD?$CD?$CD?$CD?5WinAccessBridg@ 000000018000b2b8     WinAccessBridge.obj
 0002:00002300       ??_C@_0FA@BNCMMHDE@?$FLINFO?$FN?3?5?$CD?$CD?$CD?$CD?$CD?5WinAccessBridge?3?3@ 000000018000b300     WinAccessBridge.obj
 0002:00002350       ??_C@_0EE@HJIACDJB@?$FLINFO?$FN?3?5?5?5?$CD?$CD?$CD?$CD?$CD?5WinAccessBridge@ 000000018000b350     WinAccessBridge.obj
 0002:000023a0       ??_C@_0EC@HJIAKIIH@?$FLERROR?$FN?3?5?5?5?$CD?$CD?$CD?$CD?$CD?5WinAccessBridg@ 000000018000b3a0     WinAccessBridge.obj
 0002:000023f0       ??_C@_0FF@NCBHFIIB@?$FLINFO?$FN?3?5?$CD?$CD?$CD?$CD?$CD?5WinAccessBridge?3?3@ 000000018000b3f0     WinAccessBridge.obj
 0002:00002450       ??_C@_0ED@CBAGECAG@?$FLINFO?$FN?3?5?5?5?$CD?$CD?$CD?$CD?$CD?5WinAccessBridge@ 000000018000b450     WinAccessBridge.obj
 0002:000024a0       ??_C@_0EB@NLKCNKIL@?$FLERROR?$FN?3?5?5?5?$CD?$CD?$CD?$CD?$CD?5WinAccessBridg@ 000000018000b4a0     WinAccessBridge.obj
 0002:000024f0       ??_C@_0EK@KPCBMLHL@?$FLINFO?$FN?3?5?$CD?$CD?$CD?$CD?$CD?5WinAccessBridge?3?3@ 000000018000b4f0     WinAccessBridge.obj
 0002:00002540       ??_C@_0ED@KBOKJBJ@?$FLINFO?$FN?3?5?5?5?$CD?$CD?$CD?$CD?$CD?5pkg?9?$DOrAccessibl@ 000000018000b540     WinAccessBridge.obj
 0002:00002590       ??_C@_0EE@MLCJPFKH@?$FLINFO?$FN?3?5?5?5?$CD?$CD?$CD?$CD?$CD?5WinAccessBridge@ 000000018000b590     WinAccessBridge.obj
 0002:000025e0       ??_C@_0EC@ONHLHLKJ@?$FLERROR?$FN?3?5?5?5?$CD?$CD?$CD?$CD?$CD?5WinAccessBridg@ 000000018000b5e0     WinAccessBridge.obj
 0002:00002630       ??_C@_0EI@BEINFODC@?$FLINFO?$FN?3?5?$CD?$CD?$CD?$CD?$CD?5WinAccessBridge?3?3@ 000000018000b630     WinAccessBridge.obj
 0002:00002678       ??_C@_0CN@CIJKLIHC@?$FLINFO?$FN?3?5?5?5?$CD?$CD?$CD?$CD?$CD?5hypertextInfo?4l@ 000000018000b678     WinAccessBridge.obj
 0002:000026b0       ??_C@_0EC@GJFIBKBJ@?$FLINFO?$FN?3?5?5?5?$CD?$CD?$CD?$CD?$CD?5WinAccessBridge@ 000000018000b6b0     WinAccessBridge.obj
 0002:00002700       ??_C@_0EA@ENIAHHMF@?$FLERROR?$FN?3?5?5?5?$CD?$CD?$CD?$CD?$CD?5WinAccessBridg@ 000000018000b700     WinAccessBridge.obj
 0002:00002740       ??_C@_0EI@MFFNFMHA@?$FLINFO?$FN?3?5WinAccessBridge?3?3activa@ 000000018000b740     WinAccessBridge.obj
 0002:00002790       ??_C@_0GC@OOPIFCLD@?$FLERROR?$FN?3?5?5WinAccessBridge?3?3acti@ 000000018000b790     WinAccessBridge.obj
 0002:00002800       ??_C@_0EJ@KNECEC@?$FLINFO?$FN?3?5?$CD?$CD?$CD?$CD?$CD?5WinAccessBridge?3?3@ 000000018000b800     WinAccessBridge.obj
 0002:00002850       ??_C@_0CJ@CHHBPBDA@?$FLINFO?$FN?3?5?5?5?$CD?$CD?$CD?$CD?$CD?5hypetext?5link?5c@ 000000018000b850     WinAccessBridge.obj
 0002:00002880       ??_C@_0EG@OFFPNIFM@?$FLINFO?$FN?3?5?5?$CD?$CD?$CD?$CD?$CD?5WinAccessBridge?3@ 000000018000b880     WinAccessBridge.obj
 0002:000028d0       ??_C@_0EF@CJEMCIKC@?$FLERROR?$FN?3?5?5?5?$CD?$CD?$CD?$CD?$CD?5WinAccessBridg@ 000000018000b8d0     WinAccessBridge.obj
 0002:00002920       ??_C@_0EK@KALHBKDC@?$FLINFO?$FN?3?5?$CD?$CD?$CD?$CD?$CD?5WinAccessBridge?3?3@ 000000018000b920     WinAccessBridge.obj
 0002:00002970       ??_C@_0CD@FAKLHPNN@?$FLINFO?$FN?3?5?5?5?$CD?$CD?$CD?$CD?$CD?5pkg?9?$DOrSuccess?5?$DN@ 000000018000b970     WinAccessBridge.obj
 0002:000029a0       ??_C@_0ED@CLMPFLBE@?$FLERROR?$FN?3?5?5?5?$CD?$CD?$CD?$CD?$CD?5WinAccessBridg@ 000000018000b9a0     WinAccessBridge.obj
 0002:000029f0       ??_C@_0EC@DJBOOIDG@?$FLERROR?$FN?3?5?5?$CD?$CD?$CD?$CD?$CD?5WinAccessBridge@ 000000018000b9f0     WinAccessBridge.obj
 0002:00002a40       ??_C@_0EN@IMDNGAME@?$FLINFO?$FN?3?5?$CD?$CD?$CD?$CD?$CD?5WinAccessBridge?3?3@ 000000018000ba40     WinAccessBridge.obj
 0002:00002a90       ??_C@_0CJ@LGNOCJK@?$FLINFO?$FN?3?5?5?5?$CD?$CD?$CD?$CD?$CD?5hypetext?5link?5i@ 000000018000ba90     WinAccessBridge.obj
 0002:00002ac0       ??_C@_0EM@KCINDCOI@?$FLINFO?$FN?3?5?5?5?$CD?$CD?$CD?$CD?$CD?5WinAccessBridge@ 000000018000bac0     WinAccessBridge.obj
 0002:00002b10       ??_C@_0EI@IEJDJKBK@?$FLERROR?$FN?5?5?$CD?$CD?$CD?$CD?$CD?5WinAccessBridge?3@ 000000018000bb10     WinAccessBridge.obj
 0002:00002b60       ??_C@_0EI@OHHKPFCO@?$FLINFO?$FN?3?5?$CD?$CD?$CD?$CD?$CD?5WinAccessBridge?3?3@ 000000018000bb60     WinAccessBridge.obj
 0002:00002bb0       ??_C@_0EK@CIOPKHEJ@?$FLINFO?$FN?3?5?$CD?$CD?$CD?$CD?$CD?5WinAccessBridge?3?3@ 000000018000bbb0     WinAccessBridge.obj
 0002:00002c00       ??_C@_0DC@GOKFJHHA@?$FLINFO?$FN?3?5?5?5?$CD?$CD?$CD?$CD?$CD?5keyBindings?4key@ 000000018000bc00     WinAccessBridge.obj
 0002:00002c40       ??_C@_0KM@PICKCJIM@?$FLINFO?$FN?3?5?5?5Key?5Binding?5?$CD?5?$CFd?5?5?5?5?5@ 000000018000bc40     WinAccessBridge.obj
 0002:00002cf0       ??_C@_0EE@LGIDNFJF@?$FLINFO?$FN?3?5?5?5?$CD?$CD?$CD?$CD?$CD?5WinAccessBridge@ 000000018000bcf0     WinAccessBridge.obj
 0002:00002d40       ??_C@_0EB@PIGLELIJ@?$FLINFO?$FN?3?5?5?5?$CD?$CD?$CD?$CD?$CD?5WinAccessBridge@ 000000018000bd40     WinAccessBridge.obj
 0002:00002d90       ??_C@_0EE@KBJHDGDB@?$FLINFO?$FN?3?5?$CD?$CD?$CD?$CD?$CD?5WinAccessBridge?3?3@ 000000018000bd90     WinAccessBridge.obj
 0002:00002dd8       ??_C@_0CG@JNBKIMJN@?$FLINFO?$FN?3?5?5?5?$CD?$CD?$CD?$CD?$CD?5icons?4iconsCoun@ 000000018000bdd8     WinAccessBridge.obj
 0002:00002e00       ??_C@_0DO@JGGAAEEG@?$FLINFO?$FN?3?5?5?5?$CD?$CD?$CD?$CD?$CD?5WinAccessBridge@ 000000018000be00     WinAccessBridge.obj
 0002:00002e40       ??_C@_0DM@PHFGBDGG@?$FLERROR?$FN?3?5?5?5?$CD?$CD?$CD?$CD?$CD?5WinAccessBridg@ 000000018000be40     WinAccessBridge.obj
 0002:00002e80       ??_C@_0EG@EKEEJFO@?$FLINFO?$FN?3?5?$CD?$CD?$CD?$CD?$CD?5WinAccessBridge?3?3@ 000000018000be80     WinAccessBridge.obj
 0002:00002ec8       ??_C@_0CK@COBILBN@?$FLINFO?$FN?3?5?5?5?$CD?$CD?$CD?$CD?$CD?5actions?4actions@ 000000018000bec8     WinAccessBridge.obj
 0002:00002f00       ??_C@_0EA@EKDNLNJA@?$FLINFO?$FN?3?5?5?5?$CD?$CD?$CD?$CD?$CD?5WinAccessBridge@ 000000018000bf00     WinAccessBridge.obj
 0002:00002f40       ??_C@_0DO@HNCGODDL@?$FLERROR?$FN?3?5?5?5?$CD?$CD?$CD?$CD?$CD?5WinAccessBridg@ 000000018000bf40     WinAccessBridge.obj
 0002:00002f80       ??_C@_0EH@IJHNMJPE@?$FLINFO?$FN?3?5WinAccessBridge?3?3doAcce@ 000000018000bf80     WinAccessBridge.obj
 0002:00002fd0       ??_C@_0FL@LJNDNJAB@?$FLERROR?$FN?3?5?5?5WinAccessBridge?3?3doA@ 000000018000bfd0     WinAccessBridge.obj
 0002:00003030       ??_C@_0DF@LBCGPHPD@?$FLINFO?$FN?3?5WinAccessBridge?3?3setTex@ 000000018000c030     WinAccessBridge.obj
 0002:00003068       ??_C@_0DJ@BDMKEGCI@?$FLINFO?$FN?3?5WinAccessBridge?3?3getPar@ 000000018000c068     WinAccessBridge.obj
 0002:000030b0       ??_C@_0FE@FILBCBC@?$FLINFO?$FN?3?5?5?5pkg?9?$DOvmID?3?5?$CFX?5?5?5?5?5?5?5?5@ 000000018000c0b0     WinAccessBridge.obj
 0002:00003108       ??_C@_0CG@EPJKPFNH@?$FLINFO?$FN?3?5?5?5pkg?9?$DOrAccessibleConte@ 000000018000c108     WinAccessBridge.obj
 0002:00003130       ??_C@_0DJ@LMOBJNAA@?$FLINFO?$FN?3?5WinAccessBridge?3?3getTop@ 000000018000c130     WinAccessBridge.obj
 0002:00003170       ??_C@_0EB@EGNBJNPN@?$FLINFO?$FN?3?5WinAccessBridge?3?3getPar@ 000000018000c170     WinAccessBridge.obj
 0002:000031b8       ??_C@_0DG@HMAMEAHE@?$FLINFO?$FN?3?5WinAccessBridge?3?3getObj@ 000000018000c1b8     WinAccessBridge.obj
 0002:000031f0       ??_C@_0DL@DIELJEEF@?$FLINFO?$FN?3?5WinAccessBridge?3?3getAct@ 000000018000c1f0     WinAccessBridge.obj
 0002:00003230       ??_C@_0EA@KKNJCPIF@?$FLINFO?$FN?3?5WinAccessBridge?3?3getVir@ 000000018000c230     WinAccessBridge.obj
 0002:00003270       ??_C@_0EK@LJJEDFEG@?$FLINFO?$FN?3?5?5?5?5?5WinAccessBridge?3?3ge@ 000000018000c270     WinAccessBridge.obj
 0002:000032c0       ??_C@_0DE@NGCOAPLI@?$FLINFO?$FN?3?5WinAccessBridge?3?3reques@ 000000018000c2c0     WinAccessBridge.obj
 0002:00003300       ??_C@_0EB@LDKGCIL@?$FLINFO?$FN?3?5?5?5?5?5WinAccessBridge?3?3se@ 000000018000c300     WinAccessBridge.obj
 0002:00003350       ??_C@_0EK@FKPJFOFL@?$FLINFO?$FN?3?5?5?5?5?5WinAccessBridge?3?3ge@ 000000018000c350     WinAccessBridge.obj
 0002:000033a0       ??_C@_0DP@PHLAPJAH@?$FLINFO?$FN?3?5WinAccessBridge?3?3getVis@ 000000018000c3a0     WinAccessBridge.obj
 0002:000033e0       ??_C@_0DK@FFJLHNNJ@?$FLINFO?$FN?3?5WinAccessBridge?3?3getVis@ 000000018000c3e0     WinAccessBridge.obj
 0002:00003420       ??_C@_0DM@MCJMMMCP@?$FLINFO?$FN?3?5WinAccessBridge?3?3setCar@ 000000018000c420     WinAccessBridge.obj
 0002:00003460       ??_C@_0EJ@FBPIKPOJ@?$FLINFO?$FN?3?5WinAccessBridge?3?3getAcc@ 000000018000c460     WinAccessBridge.obj
 0002:000034b0       ??_C@_0EK@DNDDFNHD@?$FLINFO?$FN?3?5?5?5charCount?3?5?$CFd?5?5?5?5?5?5?5?5@ 000000018000c4b0     WinAccessBridge.obj
 0002:00003500       ??_C@_0EG@BGFOEIHE@?$FLINFO?$FN?3?5WinAccessBridge?3?3getAcc@ 000000018000c500     WinAccessBridge.obj
 0002:00003550       ??_C@_0EK@KLCBPNFL@?$FLINFO?$FN?3?5WinAccessBridge?3?3getAcc@ 000000018000c550     WinAccessBridge.obj
 0002:000035a0       ??_C@_0EL@MJHEEFIF@?$FLINFO?$FN?3?5WinAccessBridge?3?3getAcc@ 000000018000c5a0     WinAccessBridge.obj
 0002:000035f0       ??_C@_0EF@MMEINAI@?$FLINFO?$FN?3?5WinAccessBridge?3?3getAcc@ 000000018000c5f0     WinAccessBridge.obj
 0002:00003640       ??_C@_0EA@GJMJEHDC@?$FLINFO?$FN?3?5WinAccessBridge?3?3getCar@ 000000018000c640     WinAccessBridge.obj
 0002:00003680       ??_C@_0EJ@BCHIKCEF@?$FLINFO?$FN?3?5WinAccessBridge?3?3getAcc@ 000000018000c680     WinAccessBridge.obj
 0002:000036d0       ??_C@_0EI@LCFAOBKP@?$FLINFO?$FN?3?5WinAccessBridge?3?3getAcc@ 000000018000c6d0     WinAccessBridge.obj
 0002:00003718       ??_C@_0DM@NFGOCJPM@?$FLINFO?$FN?3?5WinAccessBridge?3?3addJav@ 000000018000c718     WinAccessBridge.obj
 0002:00003758       ??_C@_0DP@PIGNLFHB@?$FLINFO?$FN?3?5?5?5?9?$DOpkgType?5?$DN?5?$CFX?0?5event@ 000000018000c758     WinAccessBridge.obj
 0002:000037a0       ??_C@_0EC@OKCIJGM@?$FLINFO?$FN?3?5in?5WinAccessBridge?3?3rem@ 000000018000c7a0     WinAccessBridge.obj
 0002:000037f0       ??_C@_0EI@HMKIAPB@?$FLINFO?$FN?3?5in?5WinAccessBridge?3?3add@ 000000018000c7f0     WinAccessBridge.obj
 0002:00003838       ??_C@_0DP@KFDABLNL@?$FLINFO?$FN?3?5?5?5?9?$DOpkgType?5?$DN?5?$CFX?0?5event@ 000000018000c838     WinAccessBridge.obj
 0002:00003880       ??_C@_0EL@BFCCGHFN@?$FLINFO?$FN?3?5in?5WinAccessBridge?3?3rem@ 000000018000c880     WinAccessBridge.obj
 0002:000038d8       ??_7type_info@@6B@         000000018000c8d8     MSVCRT:std_type_info_static.obj
 0002:000038e0       _pDefaultRawDllMain        000000018000c8e0     MSVCRT:dll_dllmain.obj
 0002:000038e0       _pRawDllMain               000000018000c8e0     MSVCRT:dll_dllmain.obj
 0002:00003900       ??_7bad_array_new_length@std@@6B@ 000000018000c900     MSVCRT:throw_bad_alloc.obj
 0002:00003910       ??_C@_0BF@KINCDENJ@bad?5array?5new?5length@ 000000018000c910     MSVCRT:throw_bad_alloc.obj
 0002:00003930       __xmm@ffffffffffffffffffffffffffffffff 000000018000c930     MSVCRT:utility.obj
 0002:00003940       _load_config_used          000000018000c940     MSVCRT:loadcfg.obj
 0002:00003b00       ??_R4exception@std@@6B@    000000018000cb00     AccessBridgeMessageQueue.obj
 0002:00003b28       ??_R3exception@std@@8      000000018000cb28     AccessBridgeMessageQueue.obj
 0002:00003b40       ??_R2exception@std@@8      000000018000cb40     AccessBridgeMessageQueue.obj
 0002:00003b50       ??_R1A@?0A@EA@exception@std@@8 000000018000cb50     AccessBridgeMessageQueue.obj
 0002:00003b78       ??_R4bad_alloc@std@@6B@    000000018000cb78     AccessBridgeMessageQueue.obj
 0002:00003ba0       ??_R3bad_alloc@std@@8      000000018000cba0     AccessBridgeMessageQueue.obj
 0002:00003bb8       ??_R2bad_alloc@std@@8      000000018000cbb8     AccessBridgeMessageQueue.obj
 0002:00003bd0       ??_R1A@?0A@EA@bad_alloc@std@@8 000000018000cbd0     AccessBridgeMessageQueue.obj
 0002:00003bf8       ??_R4type_info@@6B@        000000018000cbf8     MSVCRT:std_type_info_static.obj
 0002:00003c20       ??_R3type_info@@8          000000018000cc20     MSVCRT:std_type_info_static.obj
 0002:00003c38       ??_R2type_info@@8          000000018000cc38     MSVCRT:std_type_info_static.obj
 0002:00003c48       ??_R1A@?0A@EA@type_info@@8 000000018000cc48     MSVCRT:std_type_info_static.obj
 0002:00003c70       ??_R4bad_array_new_length@std@@6B@ 000000018000cc70     MSVCRT:throw_bad_alloc.obj
 0002:00003c98       ??_R3bad_array_new_length@std@@8 000000018000cc98     MSVCRT:throw_bad_alloc.obj
 0002:00003cb0       ??_R2bad_array_new_length@std@@8 000000018000ccb0     MSVCRT:throw_bad_alloc.obj
 0002:00003cd0       ??_R1A@?0A@EA@bad_array_new_length@std@@8 000000018000ccd0     MSVCRT:throw_bad_alloc.obj
 0002:00003cf4       __volatile_metadata        000000018000ccf4     <linker-defined>
 0002:00004078       __rtc_iaa                  000000018000d078     MSVCRT:initsect.obj
 0002:00004080       __rtc_izz                  000000018000d080     MSVCRT:initsect.obj
 0002:00004088       __rtc_taa                  000000018000d088     MSVCRT:initsect.obj
 0002:00004090       __rtc_tzz                  000000018000d090     MSVCRT:initsect.obj
 0002:000046b0       _CT??_R0?AVbad_alloc@std@@@8??0bad_alloc@std@@QEAA@AEBV01@@Z24 000000018000d6b0     AccessBridgeMessageQueue.obj
 0002:000046d8       _CT??_R0?AVexception@std@@@8??0exception@std@@QEAA@AEBV01@@Z24 000000018000d6d8     AccessBridgeMessageQueue.obj
 0002:00004700       _TI2?AVbad_alloc@std@@     000000018000d700     AccessBridgeMessageQueue.obj
 0002:00004720       _CTA2?AVbad_alloc@std@@    000000018000d720     AccessBridgeMessageQueue.obj
 0002:00004738       _TI3?AVbad_array_new_length@std@@ 000000018000d738     MSVCRT:throw_bad_alloc.obj
 0002:00004758       _CTA3?AVbad_array_new_length@std@@ 000000018000d758     MSVCRT:throw_bad_alloc.obj
 0002:00004778       _CT??_R0?AVbad_array_new_length@std@@@8??0bad_array_new_length@std@@QEAA@AEBV01@@Z24 000000018000d778     MSVCRT:throw_bad_alloc.obj
 0002:00005540       __IMPORT_DESCRIPTOR_KERNEL32 000000018000e540     kernel32:KERNEL32.dll
 0002:00005554       __IMPORT_DESCRIPTOR_USER32 000000018000e554     user32:USER32.dll
 0002:00005568       __IMPORT_DESCRIPTOR_VCRUNTIME140 000000018000e568     vcruntime:VCRUNTIME140.dll
 0002:0000557c       __IMPORT_DESCRIPTOR_api-ms-win-crt-string-l1-1-0 000000018000e57c     ucrt:api-ms-win-crt-string-l1-1-0.dll
 0002:00005590       __IMPORT_DESCRIPTOR_api-ms-win-crt-stdio-l1-1-0 000000018000e590     ucrt:api-ms-win-crt-stdio-l1-1-0.dll
 0002:000055a4       __IMPORT_DESCRIPTOR_api-ms-win-crt-environment-l1-1-0 000000018000e5a4     ucrt:api-ms-win-crt-environment-l1-1-0.dll
 0002:000055b8       __IMPORT_DESCRIPTOR_api-ms-win-crt-heap-l1-1-0 000000018000e5b8     ucrt:api-ms-win-crt-heap-l1-1-0.dll
 0002:000055cc       __IMPORT_DESCRIPTOR_api-ms-win-crt-runtime-l1-1-0 000000018000e5cc     ucrt:api-ms-win-crt-runtime-l1-1-0.dll
 0002:000055e0       __NULL_IMPORT_DESCRIPTOR   000000018000e5e0     kernel32:KERNEL32.dll
 0003:00000000       __security_cookie          000000018000f000     MSVCRT:gs_cookie.obj
 0003:00000008       __security_cookie_complement 000000018000f008     MSVCRT:gs_cookie.obj
 0003:00000010       __scrt_native_dllmain_reason 000000018000f010     MSVCRT:utility.obj
 0003:00000018       __isa_available            000000018000f018     MSVCRT:cpu_disp.obj
 0003:0000001c       __isa_enabled              000000018000f01c     MSVCRT:cpu_disp.obj
 0003:00000020       __memset_fast_string_threshold 000000018000f020     MSVCRT:cpu_disp.obj
 0003:00000028       __memset_nt_threshold      000000018000f028     MSVCRT:cpu_disp.obj
 0003:00000030       __scrt_ucrt_dll_is_in_use  000000018000f030     MSVCRT:ucrt_stubs.obj
 0003:00000038       ??_R0?AVbad_alloc@std@@@8  000000018000f038     AccessBridgeMessageQueue.obj
 0003:00000060       ??_R0?AVexception@std@@@8  000000018000f060     AccessBridgeMessageQueue.obj
 0003:00000088       ??_R0?AVbad_array_new_length@std@@@8 000000018000f088     MSVCRT:throw_bad_alloc.obj
 0003:000000b8       ??_R0?AVtype_info@@@8      000000018000f0b8     MSVCRT:std_type_info_static.obj
 0003:000000e0       ?_OptionsStorage@?1??__local_stdio_printf_options@@9@4_KA 000000018000f0e0     AccessBridgeDebug.obj
 0003:000000f0       ?theFromJavaHelloMsgID@@3IA 000000018000f0f0     AccessBridgeMessages.obj
 0003:000000f4       ?theFromWindowsHelloMsgID@@3IA 000000018000f0f4     AccessBridgeMessages.obj
 0003:000000f8       ?sendMemoryIPCLock@@3U_RTL_CRITICAL_SECTION@@A 000000018000f0f8     WinAccessBridge.obj
 0003:00000120       ?newJVMs@@3PEAPEADEA       000000018000f120     WinAccessBridge.obj
 0003:00000128       ?theWindowsAccessBridge@@3PEAVWinAccessBridge@@EA 000000018000f128     WinAccessBridge.obj
 0003:00000130       ?theDialogWindow@@3PEAUHWND__@@EA 000000018000f130     WinAccessBridge.obj
 0003:00000138       ?isVMInstanceChainInUse@@3_NA 000000018000f138     WinAccessBridge.obj
 0003:000006b0       ?__type_info_root_node@@3U__type_info_node@@A 000000018000f6b0     MSVCRT:tncleanup.obj
 0003:000006c0       ?_OptionsStorage@?1??__local_stdio_scanf_options@@9@4_KA 000000018000f6c0     MSVCRT:default_local_stdio_options.obj
 0003:000006c8       __scrt_current_native_startup_state 000000018000f6c8     MSVCRT:utility.obj
 0003:000006d0       __scrt_native_startup_lock 000000018000f6d0     MSVCRT:utility.obj
 0003:00000710       __scrt_debugger_hook_flag  000000018000f710     MSVCRT:utility_desktop.obj
 0003:00000714       __favor                    000000018000f714     MSVCRT:cpu_disp.obj
 0003:00000718       __dyn_tls_init_callback    000000018000f718     <common>

 entry point at        0001:00006b30

 Static symbols

 0000:fffed000       .debug$S                   0000000180000000     windowsaccessbridge-64.exp
 0000:fffed000       .debug$S                   0000000180000000     vcruntime:VCRUNTIME140.dll
 0000:fffed000       .debug$S                   0000000180000000     vcruntime:VCRUNTIME140.dll
 0000:fffed000       .debug$S                   0000000180000000     vcruntime:VCRUNTIME140.dll
 0000:fffed000       .debug$S                   0000000180000000     vcruntime:VCRUNTIME140.dll
 0000:fffed000       .debug$S                   0000000180000000     vcruntime:VCRUNTIME140.dll
 0000:fffed000       .debug$S                   0000000180000000     vcruntime:VCRUNTIME140.dll
 0000:fffed000       .debug$S                   0000000180000000     vcruntime:VCRUNTIME140.dll
 0000:fffed000       .debug$S                   0000000180000000     vcruntime:VCRUNTIME140.dll
 0000:fffed000       .debug$S                   0000000180000000     vcruntime:VCRUNTIME140.dll
 0000:fffed000       .debug$S                   0000000180000000     ucrt:api-ms-win-crt-environment-l1-1-0.dll
 0000:fffed000       .debug$S                   0000000180000000     ucrt:api-ms-win-crt-heap-l1-1-0.dll
 0000:fffed000       .debug$S                   0000000180000000     ucrt:api-ms-win-crt-heap-l1-1-0.dll
 0000:fffed000       .debug$S                   0000000180000000     ucrt:api-ms-win-crt-heap-l1-1-0.dll
 0000:fffed000       .debug$S                   0000000180000000     ucrt:api-ms-win-crt-runtime-l1-1-0.dll
 0000:fffed000       .debug$S                   0000000180000000     ucrt:api-ms-win-crt-runtime-l1-1-0.dll
 0000:fffed000       .debug$S                   0000000180000000     ucrt:api-ms-win-crt-runtime-l1-1-0.dll
 0000:fffed000       .debug$S                   0000000180000000     ucrt:api-ms-win-crt-runtime-l1-1-0.dll
 0000:fffed000       .debug$S                   0000000180000000     ucrt:api-ms-win-crt-runtime-l1-1-0.dll
 0000:fffed000       .debug$S                   0000000180000000     ucrt:api-ms-win-crt-runtime-l1-1-0.dll
 0000:fffed000       .debug$S                   0000000180000000     ucrt:api-ms-win-crt-runtime-l1-1-0.dll
 0000:fffed000       .debug$S                   0000000180000000     ucrt:api-ms-win-crt-runtime-l1-1-0.dll
 0000:fffed000       .debug$S                   0000000180000000     ucrt:api-ms-win-crt-runtime-l1-1-0.dll
 0000:fffed000       .debug$S                   0000000180000000     ucrt:api-ms-win-crt-runtime-l1-1-0.dll
 0000:fffed000       .debug$S                   0000000180000000     ucrt:api-ms-win-crt-runtime-l1-1-0.dll
 0000:fffed000       .debug$S                   0000000180000000     ucrt:api-ms-win-crt-runtime-l1-1-0.dll
 0000:fffed000       .debug$S                   0000000180000000     ucrt:api-ms-win-crt-stdio-l1-1-0.dll
 0000:fffed000       .debug$S                   0000000180000000     ucrt:api-ms-win-crt-stdio-l1-1-0.dll
 0000:fffed000       .debug$S                   0000000180000000     ucrt:api-ms-win-crt-stdio-l1-1-0.dll
 0000:fffed000       .debug$S                   0000000180000000     ucrt:api-ms-win-crt-stdio-l1-1-0.dll
 0000:fffed000       .debug$S                   0000000180000000     ucrt:api-ms-win-crt-stdio-l1-1-0.dll
 0000:fffed000       .debug$S                   0000000180000000     ucrt:api-ms-win-crt-stdio-l1-1-0.dll
 0000:fffed000       .debug$S                   0000000180000000     ucrt:api-ms-win-crt-string-l1-1-0.dll
 0000:fffed000       .debug$S                   0000000180000000     ucrt:api-ms-win-crt-string-l1-1-0.dll
 0000:fffed000       .debug$S                   0000000180000000     ucrt:api-ms-win-crt-string-l1-1-0.dll
 0000:fffed000       .debug$S                   0000000180000000     ucrt:api-ms-win-crt-string-l1-1-0.dll
 0000:fffed000       .debug$S                   0000000180000000     ucrt:api-ms-win-crt-string-l1-1-0.dll
 0000:fffed000       .debug$S                   0000000180000000     ucrt:api-ms-win-crt-string-l1-1-0.dll
 0000:fffed000       .debug$S                   0000000180000000     kernel32:KERNEL32.dll
 0000:fffed000       .debug$S                   0000000180000000     kernel32:KERNEL32.dll
 0000:fffed000       .debug$S                   0000000180000000     kernel32:KERNEL32.dll
 0000:fffed000       .debug$S                   0000000180000000     kernel32:KERNEL32.dll
 0000:fffed000       .debug$S                   0000000180000000     kernel32:KERNEL32.dll
 0000:fffed000       .debug$S                   0000000180000000     kernel32:KERNEL32.dll
 0000:fffed000       .debug$S                   0000000180000000     kernel32:KERNEL32.dll
 0000:fffed000       .debug$S                   0000000180000000     kernel32:KERNEL32.dll
 0000:fffed000       .debug$S                   0000000180000000     kernel32:KERNEL32.dll
 0000:fffed000       .debug$S                   0000000180000000     kernel32:KERNEL32.dll
 0000:fffed000       .debug$S                   0000000180000000     kernel32:KERNEL32.dll
 0000:fffed000       .debug$S                   0000000180000000     kernel32:KERNEL32.dll
 0000:fffed000       .debug$S                   0000000180000000     kernel32:KERNEL32.dll
 0000:fffed000       .debug$S                   0000000180000000     kernel32:KERNEL32.dll
 0000:fffed000       .debug$S                   0000000180000000     kernel32:KERNEL32.dll
 0000:fffed000       .debug$S                   0000000180000000     kernel32:KERNEL32.dll
 0000:fffed000       .debug$S                   0000000180000000     kernel32:KERNEL32.dll
 0000:fffed000       .debug$S                   0000000180000000     kernel32:KERNEL32.dll
 0000:fffed000       .debug$S                   0000000180000000     kernel32:KERNEL32.dll
 0000:fffed000       .debug$S                   0000000180000000     kernel32:KERNEL32.dll
 0000:fffed000       .debug$S                   0000000180000000     kernel32:KERNEL32.dll
 0000:fffed000       .debug$S                   0000000180000000     kernel32:KERNEL32.dll
 0000:fffed000       .debug$S                   0000000180000000     kernel32:KERNEL32.dll
 0000:fffed000       .debug$S                   0000000180000000     kernel32:KERNEL32.dll
 0000:fffed000       .debug$S                   0000000180000000     kernel32:KERNEL32.dll
 0000:fffed000       .debug$S                   0000000180000000     kernel32:KERNEL32.dll
 0000:fffed000       .debug$S                   0000000180000000     kernel32:KERNEL32.dll
 0000:fffed000       .debug$S                   0000000180000000     user32:USER32.dll
 0000:fffed000       .debug$S                   0000000180000000     user32:USER32.dll
 0000:fffed000       .debug$S                   0000000180000000     user32:USER32.dll
 0000:fffed000       .debug$S                   0000000180000000     user32:USER32.dll
 0000:fffed000       .debug$S                   0000000180000000     user32:USER32.dll
 0000:fffed000       .debug$S                   0000000180000000     user32:USER32.dll
 0000:fffed000       .debug$S                   0000000180000000     user32:USER32.dll
 0000:fffed000       .debug$S                   0000000180000000     user32:USER32.dll
 0000:fffed000       .debug$S                   0000000180000000     user32:USER32.dll
 0000:fffed000       .debug$S                   0000000180000000     user32:USER32.dll
 0000:fffed000       .debug$S                   0000000180000000     user32:USER32.dll
 0000:fffed000       .debug$S                   0000000180000000     user32:USER32.dll
 0000:fffed000       .debug$S                   0000000180000000     user32:USER32.dll
 0001:00006710       $$000000                   0000000180007710     MSVCRT:amdsecgs.obj
 0001:000067b0       $$000000                   00000001800077b0     MSVCRT:chkstk.obj
 0001:00006810       ?dllmain_crt_dispatch@@YAHQEAUHINSTANCE__@@KQEAX@Z 0000000180007810 f   MSVCRT:dll_dllmain.obj
 0001:00006860       ?dllmain_crt_process_attach@@YAHQEAUHINSTANCE__@@QEAX@Z 0000000180007860 f   MSVCRT:dll_dllmain.obj
 0001:00006978       ?dllmain_crt_process_detach@@YAH_N@Z 0000000180007978 f   MSVCRT:dll_dllmain.obj
 0001:000069fc       ?dllmain_dispatch@@YAHQEAUHINSTANCE__@@KQEAX@Z 00000001800079fc f   MSVCRT:dll_dllmain.obj
 0001:00006c80       capture_previous_context   0000000180007c80 f   MSVCRT:gs_report.obj
 0001:000075d0       $$000000                   00000001800085d0     MSVCRT:guard_dispatch.obj
 0001:000075f0       $$000000                   00000001800085f0     MSVCRT:guard_xfg_dispatch.obj
 0001:00007606       ?fin$0@?0??dllmain_crt_process_attach@@YAHQEAUHINSTANCE__@@QEAX@Z@4HA 0000000180008606 f   MSVCRT:dll_dllmain.obj
 0001:0000761d       ?fin$0@?0??dllmain_crt_process_detach@@YAH_N@Z@4HA 000000018000861d f   MSVCRT:dll_dllmain.obj
 0001:00007636       ?fin$1@?0??dllmain_crt_process_detach@@YAH_N@Z@4HA 0000000180008636 f   MSVCRT:dll_dllmain.obj
 0001:0000764a       ?filt$0@?0??dllmain_dispatch@@YAHQEAUHINSTANCE__@@KQEAX@Z@4HA 000000018000864a f   MSVCRT:dll_dllmain.obj
 0001:00007680       __scrt_is_nonwritable_in_current_image$filt$0 0000000180008680 f   MSVCRT:utility.obj
 0002:000038e8       GS_ExceptionPointers       000000018000c8e8     MSVCRT:gs_report.obj
 0002:00004098       $unwind$PrintDebugString   000000018000d098     AccessBridgeDebug.obj
 0002:000040a0       $unwind$initializeFileLogger 000000018000d0a0     AccessBridgeDebug.obj
 0002:000040b8       $unwind$finalizeFileLogger 000000018000d0b8     AccessBridgeDebug.obj
 0002:000040b8       $unwind$getTimeStamp       000000018000d0b8     AccessBridgeDebug.obj
 0002:000040b8       $unwind$?fireCaretUpdate@AccessBridgeEventHandler@@QEAAXJ_J0@Z 000000018000d0b8     AccessBridgeEventHandler.obj
 0002:000040b8       $unwind$?fireFocusGained@AccessBridgeEventHandler@@QEAAXJ_J0@Z 000000018000d0b8     AccessBridgeEventHandler.obj
 0002:000040b8       $unwind$?fireFocusLost@AccessBridgeEventHandler@@QEAAXJ_J0@Z 000000018000d0b8     AccessBridgeEventHandler.obj
 0002:000040b8       $unwind$?fireJavaShutdown@AccessBridgeEventHandler@@QEAAXJ@Z 000000018000d0b8     AccessBridgeEventHandler.obj
 0002:000040b8       $unwind$?fireMenuCanceled@AccessBridgeEventHandler@@QEAAXJ_J0@Z 000000018000d0b8     AccessBridgeEventHandler.obj
 0002:000040b8       $unwind$?fireMenuDeselected@AccessBridgeEventHandler@@QEAAXJ_J0@Z 000000018000d0b8     AccessBridgeEventHandler.obj
 0002:000040b8       $unwind$?fireMenuSelected@AccessBridgeEventHandler@@QEAAXJ_J0@Z 000000018000d0b8     AccessBridgeEventHandler.obj
 0002:000040b8       $unwind$?fireMouseClicked@AccessBridgeEventHandler@@QEAAXJ_J0@Z 000000018000d0b8     AccessBridgeEventHandler.obj
 0002:000040b8       $unwind$?fireMouseEntered@AccessBridgeEventHandler@@QEAAXJ_J0@Z 000000018000d0b8     AccessBridgeEventHandler.obj
 0002:000040b8       $unwind$?fireMouseExited@AccessBridgeEventHandler@@QEAAXJ_J0@Z 000000018000d0b8     AccessBridgeEventHandler.obj
 0002:000040b8       $unwind$?fireMousePressed@AccessBridgeEventHandler@@QEAAXJ_J0@Z 000000018000d0b8     AccessBridgeEventHandler.obj
 0002:000040b8       $unwind$?fireMouseReleased@AccessBridgeEventHandler@@QEAAXJ_J0@Z 000000018000d0b8     AccessBridgeEventHandler.obj
 0002:000040b8       $unwind$?firePopupMenuCanceled@AccessBridgeEventHandler@@QEAAXJ_J0@Z 000000018000d0b8     AccessBridgeEventHandler.obj
 0002:000040b8       $unwind$?firePopupMenuWillBecomeInvisible@AccessBridgeEventHandler@@QEAAXJ_J0@Z 000000018000d0b8     AccessBridgeEventHandler.obj
 0002:000040b8       $unwind$?firePopupMenuWillBecomeVisible@AccessBridgeEventHandler@@QEAAXJ_J0@Z 000000018000d0b8     AccessBridgeEventHandler.obj
 0002:000040b8       $unwind$?firePropertySelectionChange@AccessBridgeEventHandler@@QEAAXJ_J0@Z 000000018000d0b8     AccessBridgeEventHandler.obj
 0002:000040b8       $unwind$?firePropertyTextChange@AccessBridgeEventHandler@@QEAAXJ_J0@Z 000000018000d0b8     AccessBridgeEventHandler.obj
 0002:000040b8       $unwind$?firePropertyVisibleDataChange@AccessBridgeEventHandler@@QEAAXJ_J0@Z 000000018000d0b8     AccessBridgeEventHandler.obj
 0002:000040b8       $unwind$?initBroadcastMessageIDs@@YAHXZ 000000018000d0b8     AccessBridgeMessages.obj
 0002:000040b8       $unwind$Windows_run        000000018000d0b8     AccessBridgeWindowsEntryPoints.obj
 0002:000040b8       $unwind$addAccessibleSelectionFromContext 000000018000d0b8     AccessBridgeWindowsEntryPoints.obj
 0002:000040b8       $unwind$clearAccessibleSelectionFromContext 000000018000d0b8     AccessBridgeWindowsEntryPoints.obj
 0002:000040b8       $unwind$getVersionInfo     000000018000d0b8     AccessBridgeWindowsEntryPoints.obj
 0002:000040b8       $unwind$releaseJavaObject  000000018000d0b8     AccessBridgeWindowsEntryPoints.obj
 0002:000040b8       $unwind$removeAccessibleSelectionFromContext 000000018000d0b8     AccessBridgeWindowsEntryPoints.obj
 0002:000040b8       $unwind$selectAllAccessibleSelectionFromContext 000000018000d0b8     AccessBridgeWindowsEntryPoints.obj
 0002:000040b8       $unwind$setCaretUpdateFP   000000018000d0b8     AccessBridgeWindowsEntryPoints.obj
 0002:000040b8       $unwind$setFocusGainedFP   000000018000d0b8     AccessBridgeWindowsEntryPoints.obj
 0002:000040b8       $unwind$setFocusLostFP     000000018000d0b8     AccessBridgeWindowsEntryPoints.obj
 0002:000040b8       $unwind$setJavaShutdownFP  000000018000d0b8     AccessBridgeWindowsEntryPoints.obj
 0002:000040b8       $unwind$setMenuCanceledFP  000000018000d0b8     AccessBridgeWindowsEntryPoints.obj
 0002:000040b8       $unwind$setMenuDeselectedFP 000000018000d0b8     AccessBridgeWindowsEntryPoints.obj
 0002:000040b8       $unwind$setMenuSelectedFP  000000018000d0b8     AccessBridgeWindowsEntryPoints.obj
 0002:000040b8       $unwind$setMouseClickedFP  000000018000d0b8     AccessBridgeWindowsEntryPoints.obj
 0002:000040b8       $unwind$setMouseEnteredFP  000000018000d0b8     AccessBridgeWindowsEntryPoints.obj
 0002:000040b8       $unwind$setMouseExitedFP   000000018000d0b8     AccessBridgeWindowsEntryPoints.obj
 0002:000040b8       $unwind$setMousePressedFP  000000018000d0b8     AccessBridgeWindowsEntryPoints.obj
 0002:000040b8       $unwind$setMouseReleasedFP 000000018000d0b8     AccessBridgeWindowsEntryPoints.obj
 0002:000040b8       $unwind$setPopupMenuCanceledFP 000000018000d0b8     AccessBridgeWindowsEntryPoints.obj
 0002:000040b8       $unwind$setPopupMenuWillBecomeInvisibleFP 000000018000d0b8     AccessBridgeWindowsEntryPoints.obj
 0002:000040b8       $unwind$setPopupMenuWillBecomeVisibleFP 000000018000d0b8     AccessBridgeWindowsEntryPoints.obj
 0002:000040b8       $unwind$setPropertyActiveDescendentChangeFP 000000018000d0b8     AccessBridgeWindowsEntryPoints.obj
 0002:000040b8       $unwind$setPropertyCaretChangeFP 000000018000d0b8     AccessBridgeWindowsEntryPoints.obj
 0002:000040b8       $unwind$setPropertyChangeFP 000000018000d0b8     AccessBridgeWindowsEntryPoints.obj
 0002:000040b8       $unwind$setPropertyChildChangeFP 000000018000d0b8     AccessBridgeWindowsEntryPoints.obj
 0002:000040b8       $unwind$setPropertyDescriptionChangeFP 000000018000d0b8     AccessBridgeWindowsEntryPoints.obj
 0002:000040b8       $unwind$setPropertyNameChangeFP 000000018000d0b8     AccessBridgeWindowsEntryPoints.obj
 0002:000040b8       $unwind$setPropertySelectionChangeFP 000000018000d0b8     AccessBridgeWindowsEntryPoints.obj
 0002:000040b8       $unwind$setPropertyStateChangeFP 000000018000d0b8     AccessBridgeWindowsEntryPoints.obj
 0002:000040b8       $unwind$setPropertyTableModelChangeFP 000000018000d0b8     AccessBridgeWindowsEntryPoints.obj
 0002:000040b8       $unwind$setPropertyTextChangeFP 000000018000d0b8     AccessBridgeWindowsEntryPoints.obj
 0002:000040b8       $unwind$setPropertyValueChangeFP 000000018000d0b8     AccessBridgeWindowsEntryPoints.obj
 0002:000040b8       $unwind$setPropertyVisibleDataChangeFP 000000018000d0b8     AccessBridgeWindowsEntryPoints.obj
 0002:000040b8       $unwind$__scrt_initialize_default_local_stdio_options 000000018000d0b8     MSVCRT:default_local_stdio_options.obj
 0002:000040b8       $unwind$?dllmain_crt_dispatch@@YAHQEAUHINSTANCE__@@KQEAX@Z 000000018000d0b8     MSVCRT:dll_dllmain.obj
 0002:000040b8       $unwind$__GSHandlerCheck   000000018000d0b8     MSVCRT:gshandler.obj
 0002:000040b8       $unwind$__scrt_acquire_startup_lock 000000018000d0b8     MSVCRT:utility.obj
 0002:000040b8       $unwind$__scrt_dllmain_after_initialize_c 000000018000d0b8     MSVCRT:utility.obj
 0002:000040b8       $unwind$__scrt_dllmain_before_initialize_c 000000018000d0b8     MSVCRT:utility.obj
 0002:000040b8       $unwind$__scrt_dllmain_crt_thread_attach 000000018000d0b8     MSVCRT:utility.obj
 0002:000040b8       $unwind$__scrt_dllmain_crt_thread_detach 000000018000d0b8     MSVCRT:utility.obj
 0002:000040b8       $unwind$__scrt_dllmain_uninitialize_c 000000018000d0b8     MSVCRT:utility.obj
 0002:000040b8       $unwind$__scrt_dllmain_uninitialize_critical 000000018000d0b8     MSVCRT:utility.obj
 0002:000040c0       $unwind$fprintf            000000018000d0c0     AccessBridgeDebug.obj
 0002:000040cc       $unwind$printf             000000018000d0cc     AccessBridgeDebug.obj
 0002:000040d8       $unwind$?firePropertyActiveDescendentChange@AccessBridgeEventHandler@@QEAAXJ_J000@Z 000000018000d0d8     AccessBridgeEventHandler.obj
 0002:000040d8       $unwind$?firePropertyCaretChange@AccessBridgeEventHandler@@QEAAXJ_J0HH@Z 000000018000d0d8     AccessBridgeEventHandler.obj
 0002:000040d8       $unwind$?firePropertyChildChange@AccessBridgeEventHandler@@QEAAXJ_J000@Z 000000018000d0d8     AccessBridgeEventHandler.obj
 0002:000040d8       $unwind$?firePropertyDescriptionChange@AccessBridgeEventHandler@@QEAAXJ_J0PEAG1@Z 000000018000d0d8     AccessBridgeEventHandler.obj
 0002:000040d8       $unwind$?firePropertyNameChange@AccessBridgeEventHandler@@QEAAXJ_J0PEAG1@Z 000000018000d0d8     AccessBridgeEventHandler.obj
 0002:000040d8       $unwind$?firePropertyStateChange@AccessBridgeEventHandler@@QEAAXJ_J0PEAG1@Z 000000018000d0d8     AccessBridgeEventHandler.obj
 0002:000040d8       $unwind$?firePropertyTableModelChange@AccessBridgeEventHandler@@QEAAXJ_J0PEAG1@Z 000000018000d0d8     AccessBridgeEventHandler.obj
 0002:000040d8       $unwind$?firePropertyValueChange@AccessBridgeEventHandler@@QEAAXJ_J0PEAG1@Z 000000018000d0d8     AccessBridgeEventHandler.obj
 0002:000040d8       $unwind$?processPackage@WinAccessBridge@@QEAAXPEADJ@Z 000000018000d0d8     WinAccessBridge.obj
 0002:000040e4       $unwind$snprintf           000000018000d0e4     AccessBridgeJavaVMInstance.obj
 0002:000040f4       $unwind$??0AccessBridgeJavaVMInstance@@QEAA@PEAUHWND__@@0JPEAV0@@Z 000000018000d0f4     AccessBridgeJavaVMInstance.obj
 0002:000040f4       $unwind$?initWindow@WinAccessBridge@@QEAAHXZ 000000018000d0f4     WinAccessBridge.obj
 0002:000040fc       $unwind$??1AccessBridgeJavaVMInstance@@QEAA@XZ 000000018000d0fc     AccessBridgeJavaVMInstance.obj
 0002:000040fc       $unwind$??0bad_alloc@std@@QEAA@AEBV01@@Z 000000018000d0fc     AccessBridgeMessageQueue.obj
 0002:000040fc       $unwind$??0exception@std@@QEAA@AEBV01@@Z 000000018000d0fc     AccessBridgeMessageQueue.obj
 0002:000040fc       $unwind$getTopLevelHWND    000000018000d0fc     AccessBridgeWindowsEntryPoints.obj
 0002:000040fc       $unwind$DllMain            000000018000d0fc     WinAccessBridge.obj
 0002:000040fc       $unwind$__raise_securityfailure 000000018000d0fc     MSVCRT:gs_report.obj
 0002:000040fc       $unwind$??2@YAPEAX_K@Z     000000018000d0fc     MSVCRT:new_scalar.obj
 0002:000040fc       $unwind$??_Gtype_info@@UEAAPEAXI@Z 000000018000d0fc     MSVCRT:std_type_info_static.obj
 0002:000040fc       $unwind$??0bad_array_new_length@std@@QEAA@AEBV01@@Z 000000018000d0fc     MSVCRT:throw_bad_alloc.obj
 0002:000040fc       $unwind$__scrt_initialize_crt 000000018000d0fc     MSVCRT:utility.obj
 0002:000040fc       $unwind$__scrt_initialize_onexit_tables 000000018000d0fc     MSVCRT:utility.obj
 0002:000040fc       $unwind$__scrt_release_startup_lock 000000018000d0fc     MSVCRT:utility.obj
 0002:000040fc       $unwind$__scrt_uninitialize_crt 000000018000d0fc     MSVCRT:utility.obj
 0002:00004104       $unwind$?initiateIPC@AccessBridgeJavaVMInstance@@QEAA_JXZ 000000018000d104     AccessBridgeJavaVMInstance.obj
 0002:0000411c       $unwind$?sendPackage@AccessBridgeJavaVMInstance@@QEAA_JPEADJ@Z 000000018000d11c     AccessBridgeJavaVMInstance.obj
 0002:00004124       $unwind$?sendMemoryPackage@AccessBridgeJavaVMInstance@@QEAAHPEADJ@Z 000000018000d124     AccessBridgeJavaVMInstance.obj
 0002:0000413c       $unwind$?findABJavaVMInstanceFromJavaHWND@AccessBridgeJavaVMInstance@@QEAAPEAV1@PEAUHWND__@@@Z 000000018000d13c     AccessBridgeJavaVMInstance.obj
 0002:0000413c       $unwind$?findAccessBridgeWindow@AccessBridgeJavaVMInstance@@QEAAPEAUHWND__@@J@Z 000000018000d13c     AccessBridgeJavaVMInstance.obj
 0002:0000413c       $unwind$??_Gbad_alloc@std@@UEAAPEAXI@Z 000000018000d13c     AccessBridgeMessageQueue.obj
 0002:0000413c       $unwind$??_Gexception@std@@UEAAPEAXI@Z 000000018000d13c     AccessBridgeMessageQueue.obj
 0002:0000413c       $unwind$??0WinAccessBridge@@QEAA@PEAUHINSTANCE__@@@Z 000000018000d13c     WinAccessBridge.obj
 0002:0000413c       $unwind$??1WinAccessBridge@@QEAA@XZ 000000018000d13c     WinAccessBridge.obj
 0002:0000413c       $unwind$?sendMemoryPackage@WinAccessBridge@@QEAAHPEADJPEAUHWND__@@@Z 000000018000d13c     WinAccessBridge.obj
 0002:0000413c       $unwind$_RTC_Initialize    000000018000d13c     MSVCRT:initsect.obj
 0002:0000413c       $unwind$_RTC_Terminate     000000018000d13c     MSVCRT:initsect.obj
 0002:0000413c       $unwind$??_Gbad_array_new_length@std@@UEAAPEAXI@Z 000000018000d13c     MSVCRT:throw_bad_alloc.obj
 0002:00004148       $unwind$??0AccessBridgeQueueElement@@QEAA@PEADH@Z 000000018000d148     AccessBridgeMessageQueue.obj
 0002:00004154       $unwind$?add@AccessBridgeMessageQueue@@QEAA?AW4QueueReturns@@PEAVAccessBridgeQueueElement@@@Z 000000018000d154     AccessBridgeMessageQueue.obj
 0002:00004154       $unwind$?remove@AccessBridgeMessageQueue@@QEAA?AW4QueueReturns@@PEAPEAVAccessBridgeQueueElement@@@Z 000000018000d154     AccessBridgeMessageQueue.obj
 0002:00004154       $unwind$isSameObject       000000018000d154     AccessBridgeWindowsEntryPoints.obj
 0002:00004154       $unwind$?JavaVMDestroyed@WinAccessBridge@@QEAAXPEAUHWND__@@@Z 000000018000d154     WinAccessBridge.obj
 0002:00004154       $unwind$?preProcessPackage@WinAccessBridge@@QEAAXPEADJ@Z 000000018000d154     WinAccessBridge.obj
 0002:00004154       $unwind$?queuePackage@WinAccessBridge@@QEAAHPEADJ@Z 000000018000d154     WinAccessBridge.obj
 0002:00004154       $unwind$AccessBridgeDialogProc 000000018000d154     WinAccessBridge.obj
 0002:00004154       $unwind$_DllMainCRTStartup 000000018000d154     MSVCRT:dll_dllmain.obj
 0002:00004164       $unwind$doAccessibleActions 000000018000d164     AccessBridgeWindowsEntryPoints.obj
 0002:00004164       $unwind$getAccessibleContextAt 000000018000d164     AccessBridgeWindowsEntryPoints.obj
 0002:00004164       $unwind$getAccessibleHyperlink 000000018000d164     AccessBridgeWindowsEntryPoints.obj
 0002:00004164       $unwind$getAccessibleHypertextExt 000000018000d164     AccessBridgeWindowsEntryPoints.obj
 0002:00004164       $unwind$getAccessibleTableCellInfo 000000018000d164     AccessBridgeWindowsEntryPoints.obj
 0002:00004164       $unwind$getAccessibleTableColumnSelections 000000018000d164     AccessBridgeWindowsEntryPoints.obj
 0002:00004164       $unwind$getAccessibleTableIndex 000000018000d164     AccessBridgeWindowsEntryPoints.obj
 0002:00004164       $unwind$getAccessibleTableRowSelections 000000018000d164     AccessBridgeWindowsEntryPoints.obj
 0002:00004164       $unwind$getAccessibleTextAttributes 000000018000d164     AccessBridgeWindowsEntryPoints.obj
 0002:00004164       $unwind$getAccessibleTextInfo 000000018000d164     AccessBridgeWindowsEntryPoints.obj
 0002:00004164       $unwind$getAccessibleTextItems 000000018000d164     AccessBridgeWindowsEntryPoints.obj
 0002:00004164       $unwind$getAccessibleTextLineBounds 000000018000d164     AccessBridgeWindowsEntryPoints.obj
 0002:00004164       $unwind$getAccessibleTextRect 000000018000d164     AccessBridgeWindowsEntryPoints.obj
 0002:00004164       $unwind$getCaretLocation   000000018000d164     AccessBridgeWindowsEntryPoints.obj
 0002:00004164       $unwind$getCurrentAccessibleValueFromContext 000000018000d164     AccessBridgeWindowsEntryPoints.obj
 0002:00004164       $unwind$getMaximumAccessibleValueFromContext 000000018000d164     AccessBridgeWindowsEntryPoints.obj
 0002:00004164       $unwind$getMinimumAccessibleValueFromContext 000000018000d164     AccessBridgeWindowsEntryPoints.obj
 0002:00004164       $unwind$getVirtualAccessibleName 000000018000d164     AccessBridgeWindowsEntryPoints.obj
 0002:00004164       $unwind$getVisibleChildren 000000018000d164     AccessBridgeWindowsEntryPoints.obj
 0002:00004164       $unwind$selectTextRange    000000018000d164     AccessBridgeWindowsEntryPoints.obj
 0002:0000416c       $unwind$getAccessibleTextRange 000000018000d16c     AccessBridgeWindowsEntryPoints.obj
 0002:0000416c       $unwind$getTextAttributesInRange 000000018000d16c     AccessBridgeWindowsEntryPoints.obj
 0002:0000416c       $unwind$?__scrt_throw_std_bad_alloc@@YAXXZ 000000018000d16c     MSVCRT:throw_bad_alloc.obj
 0002:0000416c       $unwind$?__scrt_throw_std_bad_array_new_length@@YAXXZ 000000018000d16c     MSVCRT:throw_bad_alloc.obj
 0002:00004174       $unwind$?rendezvousWithNewJavaDLL@WinAccessBridge@@QEAA_JPEAUHWND__@@J@Z 000000018000d174     WinAccessBridge.obj
 0002:00004184       $unwind$?sendPackage@WinAccessBridge@@QEAAXPEADJPEAUHWND__@@@Z 000000018000d184     WinAccessBridge.obj
 0002:0000418c       $unwind$?receiveAQueuedPackage@WinAccessBridge@@QEAAHXZ 000000018000d18c     WinAccessBridge.obj
 0002:0000419c       $unwind$?getHWNDFromAccessibleContext@WinAccessBridge@@QEAAPEAUHWND__@@J_J@Z 000000018000d19c     WinAccessBridge.obj
 0002:0000419c       $unwind$?releaseJavaObject@WinAccessBridge@@QEAAXJ_J@Z 000000018000d19c     WinAccessBridge.obj
 0002:0000419c       $unwind$?requestFocus@WinAccessBridge@@QEAAHJ_J@Z 000000018000d19c     WinAccessBridge.obj
 0002:000041b0       $unwind$?getAccessibleTextSelectionInfo@WinAccessBridge@@QEAAHJ_JPEAUAccessibleTextSelectionInfoTag@@@Z 000000018000d1b0     WinAccessBridge.obj
 0002:000041b0       $unwind$?getVersionInfo@WinAccessBridge@@QEAAHJPEAUAccessBridgeVersionInfoTag@@@Z 000000018000d1b0     WinAccessBridge.obj
 0002:000041c8       $unwind$?isJavaWindow@WinAccessBridge@@QEAAHPEAUHWND__@@@Z 000000018000d1c8     WinAccessBridge.obj
 0002:000041dc       $unwind$?getAccessibleContextFromHWND@WinAccessBridge@@QEAAHPEAUHWND__@@PEAJPEA_J@Z 000000018000d1dc     WinAccessBridge.obj
 0002:000041f4       $unwind$?activateAccessibleHyperlink@WinAccessBridge@@QEAAHJ_J0@Z 000000018000d1f4     WinAccessBridge.obj
 0002:000041f4       $unwind$?isSameObject@WinAccessBridge@@QEAAHJ_J0@Z 000000018000d1f4     WinAccessBridge.obj
 0002:0000420c       $unwind$?getVirtualAccessibleName@WinAccessBridge@@QEAAHJ_JPEAGH@Z 000000018000d20c     WinAccessBridge.obj
 0002:0000420c       $unwind$?setTextContents@WinAccessBridge@@QEAAHJ_JPEBG@Z 000000018000d20c     WinAccessBridge.obj
 0002:00004224       $unwind$?getParentWithRole@WinAccessBridge@@QEAA_JJ_JPEBG@Z 000000018000d224     WinAccessBridge.obj
 0002:00004224       $unwind$?getParentWithRoleElseRoot@WinAccessBridge@@QEAA_JJ_JPEBG@Z 000000018000d224     WinAccessBridge.obj
 0002:0000423c       $unwind$?getAccessibleParentFromContext@WinAccessBridge@@QEAA_JJ_J@Z 000000018000d23c     WinAccessBridge.obj
 0002:0000423c       $unwind$?getActiveDescendent@WinAccessBridge@@QEAA_JJ_J@Z 000000018000d23c     WinAccessBridge.obj
 0002:0000423c       $unwind$?getObjectDepth@WinAccessBridge@@QEAAHJ_J@Z 000000018000d23c     WinAccessBridge.obj
 0002:0000423c       $unwind$?getTopLevelObject@WinAccessBridge@@QEAA_JJ_J@Z 000000018000d23c     WinAccessBridge.obj
 0002:0000423c       $unwind$?getVisibleChildrenCount@WinAccessBridge@@QEAAHJ_J@Z 000000018000d23c     WinAccessBridge.obj
 0002:00004250       $unwind$?getAccessibleContextAt@WinAccessBridge@@QEAAHJ_JHHPEA_J@Z 000000018000d250     WinAccessBridge.obj
 0002:00004264       $unwind$?getAccessibleContextWithFocus@WinAccessBridge@@QEAAHPEAUHWND__@@PEAJPEA_J@Z 000000018000d264     WinAccessBridge.obj
 0002:00004264       $unwind$?getAccessibleTableColumn@WinAccessBridge@@QEAAHJ_JH@Z 000000018000d264     WinAccessBridge.obj
 0002:00004264       $unwind$?getAccessibleTableRow@WinAccessBridge@@QEAAHJ_JH@Z 000000018000d264     WinAccessBridge.obj
 0002:0000427c       $unwind$?getAccessibleContextInfo@WinAccessBridge@@QEAAHJ_JPEAUAccessibleContextInfoTag@@@Z 000000018000d27c     WinAccessBridge.obj
 0002:00004294       $unwind$?getAccessibleChildFromContext@WinAccessBridge@@QEAA_JJ_JH@Z 000000018000d294     WinAccessBridge.obj
 0002:000042a8       $unwind$?getAccessibleTableColumnHeader@WinAccessBridge@@QEAAHJ_JPEAUAccessibleTableInfoTag@@@Z 000000018000d2a8     WinAccessBridge.obj
 0002:000042a8       $unwind$?getAccessibleTableInfo@WinAccessBridge@@QEAAHJ_JPEAUAccessibleTableInfoTag@@@Z 000000018000d2a8     WinAccessBridge.obj
 0002:000042a8       $unwind$?getAccessibleTableRowHeader@WinAccessBridge@@QEAAHJ_JPEAUAccessibleTableInfoTag@@@Z 000000018000d2a8     WinAccessBridge.obj
 0002:000042c0       $unwind$?getAccessibleTableCellInfo@WinAccessBridge@@QEAAHJ_JHHPEAUAccessibleTableCellInfoTag@@@Z 000000018000d2c0     WinAccessBridge.obj
 0002:000042dc       $unwind$?getAccessibleTableColumnDescription@WinAccessBridge@@QEAA_JJ_JH@Z 000000018000d2dc     WinAccessBridge.obj
 0002:000042dc       $unwind$?getAccessibleTableRowDescription@WinAccessBridge@@QEAA_JJ_JH@Z 000000018000d2dc     WinAccessBridge.obj
 0002:000042dc       $unwind$?getAccessibleTextLineBounds@WinAccessBridge@@QEAAHJ_JHPEAH1@Z 000000018000d2dc     WinAccessBridge.obj
 0002:000042f4       $unwind$?getAccessibleHyperlinkCount@WinAccessBridge@@QEAAHJ_J@Z 000000018000d2f4     WinAccessBridge.obj
 0002:000042f4       $unwind$?getAccessibleTableColumnSelectionCount@WinAccessBridge@@QEAAHJ_J@Z 000000018000d2f4     WinAccessBridge.obj
 0002:000042f4       $unwind$?getAccessibleTableRowSelectionCount@WinAccessBridge@@QEAAHJ_J@Z 000000018000d2f4     WinAccessBridge.obj
 0002:000042f4       $unwind$?setCaretPosition@WinAccessBridge@@QEAAHJ_JH@Z 000000018000d2f4     WinAccessBridge.obj
 0002:00004308       $unwind$?getAccessibleHypertextLinkIndex@WinAccessBridge@@QEAAHJ_JH@Z 000000018000d308     WinAccessBridge.obj
 0002:00004308       $unwind$?isAccessibleTableColumnSelected@WinAccessBridge@@QEAAHJ_JH@Z 000000018000d308     WinAccessBridge.obj
 0002:00004308       $unwind$?isAccessibleTableRowSelected@WinAccessBridge@@QEAAHJ_JH@Z 000000018000d308     WinAccessBridge.obj
 0002:00004320       $unwind$?getAccessibleTableColumnSelections@WinAccessBridge@@QEAAHJ_JHPEAH@Z 000000018000d320     WinAccessBridge.obj
 0002:00004320       $unwind$?getAccessibleTableRowSelections@WinAccessBridge@@QEAAHJ_JHPEAH@Z 000000018000d320     WinAccessBridge.obj
 0002:0000433c       $unwind$?getAccessibleTableIndex@WinAccessBridge@@QEAAHJ_JHH@Z 000000018000d33c     WinAccessBridge.obj
 0002:00004354       $unwind$?getAccessibleRelationSet@WinAccessBridge@@QEAAHJ_JPEAUAccessibleRelationSetInfoTag@@@Z 000000018000d354     WinAccessBridge.obj
 0002:0000436c       $unwind$?getAccessibleHypertext@WinAccessBridge@@QEAAHJ_JPEAUAccessibleHypertextInfoTag@@@Z 000000018000d36c     WinAccessBridge.obj
 0002:00004384       $unwind$?getAccessibleHypertextExt@WinAccessBridge@@QEAAHJ_JHPEAUAccessibleHypertextInfoTag@@@Z 000000018000d384     WinAccessBridge.obj
 0002:000043a0       $unwind$?getAccessibleHyperlink@WinAccessBridge@@QEAAHJ_JHPEAUAccessibleHyperlinkInfoTag@@@Z 000000018000d3a0     WinAccessBridge.obj
 0002:000043bc       $unwind$?getAccessibleKeyBindings@WinAccessBridge@@QEAAHJ_JPEAUAccessibleKeyBindingsTag@@@Z 000000018000d3bc     WinAccessBridge.obj
 0002:000043d8       $unwind$?getAccessibleIcons@WinAccessBridge@@QEAAHJ_JPEAUAccessibleIconsTag@@@Z 000000018000d3d8     WinAccessBridge.obj
 0002:000043f0       $unwind$?getAccessibleActions@WinAccessBridge@@QEAAHJ_JPEAUAccessibleActionsTag@@@Z 000000018000d3f0     WinAccessBridge.obj
 0002:00004408       $unwind$?doAccessibleActions@WinAccessBridge@@QEAAHJ_JPEAUAccessibleActionsToDoTag@@PEAH@Z 000000018000d408     WinAccessBridge.obj
 0002:00004424       $unwind$?getAccessibleTextInfo@WinAccessBridge@@QEAAHJ_JPEAUAccessibleTextInfoTag@@HH@Z 000000018000d424     WinAccessBridge.obj
 0002:00004424       $unwind$?getAccessibleTextRect@WinAccessBridge@@QEAAHJ_JPEAUAccessibleTextRectInfoTag@@H@Z 000000018000d424     WinAccessBridge.obj
 0002:00004424       $unwind$?getCaretLocation@WinAccessBridge@@QEAAHJ_JPEAUAccessibleTextRectInfoTag@@H@Z 000000018000d424     WinAccessBridge.obj
 0002:00004438       $unwind$?getAccessibleTextItems@WinAccessBridge@@QEAAHJ_JPEAUAccessibleTextItemsInfoTag@@H@Z 000000018000d438     WinAccessBridge.obj
 0002:00004450       $unwind$?getAccessibleTextAttributes@WinAccessBridge@@QEAAHJ_JHPEAUAccessibleTextAttributesInfoTag@@@Z 000000018000d450     WinAccessBridge.obj
 0002:00004468       $unwind$?getAccessibleTextRange@WinAccessBridge@@QEAAHJ_JHHPEAGF@Z 000000018000d468     WinAccessBridge.obj
 0002:00004480       $unwind$?getCurrentAccessibleValueFromContext@WinAccessBridge@@QEAAHJ_JPEAGF@Z 000000018000d480     WinAccessBridge.obj
 0002:00004480       $unwind$?getMaximumAccessibleValueFromContext@WinAccessBridge@@QEAAHJ_JPEAGF@Z 000000018000d480     WinAccessBridge.obj
 0002:00004480       $unwind$?getMinimumAccessibleValueFromContext@WinAccessBridge@@QEAAHJ_JPEAGF@Z 000000018000d480     WinAccessBridge.obj
 0002:00004498       $unwind$?addAccessibleSelectionFromContext@WinAccessBridge@@QEAAXJ_JH@Z 000000018000d498     WinAccessBridge.obj
 0002:00004498       $unwind$?getAccessibleSelectionCountFromContext@WinAccessBridge@@QEAAHJ_J@Z 000000018000d498     WinAccessBridge.obj
 0002:00004498       $unwind$?removeAccessibleSelectionFromContext@WinAccessBridge@@QEAAXJ_JH@Z 000000018000d498     WinAccessBridge.obj
 0002:000044a8       $unwind$?clearAccessibleSelectionFromContext@WinAccessBridge@@QEAAXJ_J@Z 000000018000d4a8     WinAccessBridge.obj
 0002:000044a8       $unwind$?selectAllAccessibleSelectionFromContext@WinAccessBridge@@QEAAXJ_J@Z 000000018000d4a8     WinAccessBridge.obj
 0002:000044b8       $unwind$?getAccessibleSelectionFromContext@WinAccessBridge@@QEAA_JJ_JH@Z 000000018000d4b8     WinAccessBridge.obj
 0002:000044c8       $unwind$?isAccessibleChildSelectedFromContext@WinAccessBridge@@QEAAHJ_JH@Z 000000018000d4c8     WinAccessBridge.obj
 0002:000044dc       $unwind$?addAccessibilityEventNotification@WinAccessBridge@@QEAAX_J@Z 000000018000d4dc     WinAccessBridge.obj
 0002:000044dc       $unwind$?addJavaEventNotification@WinAccessBridge@@QEAAX_J@Z 000000018000d4dc     WinAccessBridge.obj
 0002:000044dc       $unwind$?removeAccessibilityEventNotification@WinAccessBridge@@QEAAX_J@Z 000000018000d4dc     WinAccessBridge.obj
 0002:000044dc       $unwind$?removeJavaEventNotification@WinAccessBridge@@QEAAX_J@Z 000000018000d4dc     WinAccessBridge.obj
 0002:000044f0       $unwind$?selectTextRange@WinAccessBridge@@QEAAHJ_JHH@Z 000000018000d4f0     WinAccessBridge.obj
 0002:00004504       $unwind$?getTextAttributesInRange@WinAccessBridge@@QEAAHJ_JHHPEAUAccessibleTextAttributesInfoTag@@PEAF@Z 000000018000d504     WinAccessBridge.obj
 0002:00004524       $unwind$?getVisibleChildren@WinAccessBridge@@QEAAHJ_JHPEAUVisibleChildenInfoTag@@@Z 000000018000d524     WinAccessBridge.obj
 0002:0000453c       $unwind$__GSHandlerCheckCommon 000000018000d53c     MSVCRT:gshandler.obj
 0002:00004548       $xdatasym                  000000018000d548     MSVCRT:amdsecgs.obj
 0002:00004550       $xdatasym                  000000018000d550     MSVCRT:chkstk.obj
 0002:00004558       $unwind$?dllmain_crt_process_attach@@YAHQEAUHINSTANCE__@@QEAX@Z 000000018000d558     MSVCRT:dll_dllmain.obj
 0002:00004594       $unwind$?fin$0@?0??dllmain_crt_process_attach@@YAHQEAUHINSTANCE__@@QEAX@Z@4HA 000000018000d594     MSVCRT:dll_dllmain.obj
 0002:00004594       $unwind$?fin$0@?0??dllmain_crt_process_detach@@YAH_N@Z@4HA 000000018000d594     MSVCRT:dll_dllmain.obj
 0002:00004594       $unwind$?fin$1@?0??dllmain_crt_process_detach@@YAH_N@Z@4HA 000000018000d594     MSVCRT:dll_dllmain.obj
 0002:0000459c       $unwind$?dllmain_crt_process_detach@@YAH_N@Z 000000018000d59c     MSVCRT:dll_dllmain.obj
 0002:000045f0       $unwind$?dllmain_dispatch@@YAHQEAUHINSTANCE__@@KQEAX@Z 000000018000d5f0     MSVCRT:dll_dllmain.obj
 0002:00004618       $unwind$?filt$0@?0??dllmain_dispatch@@YAHQEAUHINSTANCE__@@KQEAX@Z@4HA 000000018000d618     MSVCRT:dll_dllmain.obj
 0002:00004620       $unwind$__report_gsfailure 000000018000d620     MSVCRT:gs_report.obj
 0002:00004628       $unwind$capture_previous_context 000000018000d628     MSVCRT:gs_report.obj
 0002:00004634       $unwind$__security_init_cookie 000000018000d634     MSVCRT:gs_support.obj
 0002:00004640       $unwind$__scrt_is_nonwritable_in_current_image 000000018000d640     MSVCRT:utility.obj
 0002:00004660       $unwind$__scrt_is_nonwritable_in_current_image$filt$0 000000018000d660     MSVCRT:utility.obj
 0002:00004668       $unwind$__scrt_dllmain_exception_filter 000000018000d668     MSVCRT:utility.obj
 0002:0000467c       $unwind$__scrt_fastfail    000000018000d67c     MSVCRT:utility_desktop.obj
 0002:0000468c       $unwind$__isa_available_init 000000018000d68c     MSVCRT:cpu_disp.obj
 0002:000046a0       $xdatasym                  000000018000d6a0     MSVCRT:guard_dispatch.obj
 0002:000046a8       $xdatasym                  000000018000d6a8     MSVCRT:guard_xfg_dispatch.obj
 0002:000047a0       .edata                     000000018000d7a0     windowsaccessbridge-64.exp
 0002:000047c8       rgpv                       000000018000d7c8     windowsaccessbridge-64.exp
 0002:0000494c       rgszName                   000000018000d94c     windowsaccessbridge-64.exp
 0002:00004ad0       rgwOrd                     000000018000dad0     windowsaccessbridge-64.exp
 0002:00004b92       szName                     000000018000db92     windowsaccessbridge-64.exp
 0002:00004bad       $N00001                    000000018000dbad     windowsaccessbridge-64.exp
 0002:00004bb9       $N00002                    000000018000dbb9     windowsaccessbridge-64.exp
 0002:00004bd5       $N00003                    000000018000dbd5     windowsaccessbridge-64.exp
 0002:00004bf7       $N00004                    000000018000dbf7     windowsaccessbridge-64.exp
 0002:00004c1b       $N00005                    000000018000dc1b     windowsaccessbridge-64.exp
 0002:00004c2f       $N00006                    000000018000dc2f     windowsaccessbridge-64.exp
 0002:00004c44       $N00007                    000000018000dc44     windowsaccessbridge-64.exp
 0002:00004c62       $N00008                    000000018000dc62     windowsaccessbridge-64.exp
 0002:00004c79       $N00009                    000000018000dc79     windowsaccessbridge-64.exp
 0002:00004c96       $N00010                    000000018000dc96     windowsaccessbridge-64.exp
 0002:00004caf       $N00011                    000000018000dcaf     windowsaccessbridge-64.exp
 0002:00004ccd       $N00012                    000000018000dccd     windowsaccessbridge-64.exp
 0002:00004ce4       $N00013                    000000018000dce4     windowsaccessbridge-64.exp
 0002:00004d00       $N00014                    000000018000dd00     windowsaccessbridge-64.exp
 0002:00004d17       $N00015                    000000018000dd17     windowsaccessbridge-64.exp
 0002:00004d31       $N00016                    000000018000dd31     windowsaccessbridge-64.exp
 0002:00004d51       $N00017                    000000018000dd51     windowsaccessbridge-64.exp
 0002:00004d64       $N00018                    000000018000dd64     windowsaccessbridge-64.exp
 0002:00004d7d       $N00019                    000000018000dd7d     windowsaccessbridge-64.exp
 0002:00004d9c       $N00020                    000000018000dd9c     windowsaccessbridge-64.exp
 0002:00004db5       $N00021                    000000018000ddb5     windowsaccessbridge-64.exp
 0002:00004ddc       $N00022                    000000018000dddc     windowsaccessbridge-64.exp
 0002:00004dfe       $N00023                    000000018000ddfe     windowsaccessbridge-64.exp
 0002:00004e19       $N00024                    000000018000de19     windowsaccessbridge-64.exp
 0002:00004e32       $N00025                    000000018000de32     windowsaccessbridge-64.exp
 0002:00004e56       $N00026                    000000018000de56     windowsaccessbridge-64.exp
 0002:00004e75       $N00027                    000000018000de75     windowsaccessbridge-64.exp
 0002:00004e9c       $N00028                    000000018000de9c     windowsaccessbridge-64.exp
 0002:00004ebf       $N00029                    000000018000debf     windowsaccessbridge-64.exp
 0002:00004ed7       $N00030                    000000018000ded7     windowsaccessbridge-64.exp
 0002:00004eee       $N00031                    000000018000deee     windowsaccessbridge-64.exp
 0002:00004f04       $N00032                    000000018000df04     windowsaccessbridge-64.exp
 0002:00004f25       $N00033                    000000018000df25     windowsaccessbridge-64.exp
 0002:00004f41       $N00034                    000000018000df41     windowsaccessbridge-64.exp
 0002:00004f65       $N00035                    000000018000df65     windowsaccessbridge-64.exp
 0002:00004f85       $N00036                    000000018000df85     windowsaccessbridge-64.exp
 0002:00004fa1       $N00037                    000000018000dfa1     windowsaccessbridge-64.exp
 0002:00004fb7       $N00038                    000000018000dfb7     windowsaccessbridge-64.exp
 0002:00004fce       $N00039                    000000018000dfce     windowsaccessbridge-64.exp
 0002:00004fea       $N00040                    000000018000dfea     windowsaccessbridge-64.exp
 0002:00005001       $N00041                    000000018000e001     windowsaccessbridge-64.exp
 0002:00005017       $N00042                    000000018000e017     windowsaccessbridge-64.exp
 0002:00005036       $N00043                    000000018000e036     windowsaccessbridge-64.exp
 0002:0000504a       $N00044                    000000018000e04a     windowsaccessbridge-64.exp
 0002:0000505b       $N00045                    000000018000e05b     windowsaccessbridge-64.exp
 0002:00005080       $N00046                    000000018000e080     windowsaccessbridge-64.exp
 0002:00005091       $N00047                    000000018000e091     windowsaccessbridge-64.exp
 0002:000050ae       $N00048                    000000018000e0ae     windowsaccessbridge-64.exp
 0002:000050d3       $N00049                    000000018000e0d3     windowsaccessbridge-64.exp
 0002:000050f8       $N00050                    000000018000e0f8     windowsaccessbridge-64.exp
 0002:00005107       $N00051                    000000018000e107     windowsaccessbridge-64.exp
 0002:00005119       $N00052                    000000018000e119     windowsaccessbridge-64.exp
 0002:00005133       $N00053                    000000018000e133     windowsaccessbridge-64.exp
 0002:0000514c       $N00054                    000000018000e14c     windowsaccessbridge-64.exp
 0002:0000515e       $N00055                    000000018000e15e     windowsaccessbridge-64.exp
 0002:0000516d       $N00056                    000000018000e16d     windowsaccessbridge-64.exp
 0002:00005186       $N00057                    000000018000e186     windowsaccessbridge-64.exp
 0002:00005199       $N00058                    000000018000e199     windowsaccessbridge-64.exp
 0002:000051b1       $N00059                    000000018000e1b1     windowsaccessbridge-64.exp
 0002:000051d6       $N00060                    000000018000e1d6     windowsaccessbridge-64.exp
 0002:000051f6       $N00061                    000000018000e1f6     windowsaccessbridge-64.exp
 0002:00005213       $N00062                    000000018000e213     windowsaccessbridge-64.exp
 0002:00005220       $N00063                    000000018000e220     windowsaccessbridge-64.exp
 0002:0000522d       $N00064                    000000018000e22d     windowsaccessbridge-64.exp
 0002:0000523f       $N00065                    000000018000e23f     windowsaccessbridge-64.exp
 0002:00005264       $N00066                    000000018000e264     windowsaccessbridge-64.exp
 0002:00005271       $N00067                    000000018000e271     windowsaccessbridge-64.exp
 0002:00005299       $N00068                    000000018000e299     windowsaccessbridge-64.exp
 0002:000052a9       $N00069                    000000018000e2a9     windowsaccessbridge-64.exp
 0002:000052ba       $N00070                    000000018000e2ba     windowsaccessbridge-64.exp
 0002:000052cb       $N00071                    000000018000e2cb     windowsaccessbridge-64.exp
 0002:000052dc       $N00072                    000000018000e2dc     windowsaccessbridge-64.exp
 0002:000052eb       $N00073                    000000018000e2eb     windowsaccessbridge-64.exp
 0002:000052fd       $N00074                    000000018000e2fd     windowsaccessbridge-64.exp
 0002:0000530f       $N00075                    000000018000e30f     windowsaccessbridge-64.exp
 0002:00005323       $N00076                    000000018000e323     windowsaccessbridge-64.exp
 0002:00005335       $N00077                    000000018000e335     windowsaccessbridge-64.exp
 0002:00005347       $N00078                    000000018000e347     windowsaccessbridge-64.exp
 0002:00005359       $N00079                    000000018000e359     windowsaccessbridge-64.exp
 0002:0000536a       $N00080                    000000018000e36a     windowsaccessbridge-64.exp
 0002:0000537c       $N00081                    000000018000e37c     windowsaccessbridge-64.exp
 0002:0000538f       $N00082                    000000018000e38f     windowsaccessbridge-64.exp
 0002:000053a6       $N00083                    000000018000e3a6     windowsaccessbridge-64.exp
 0002:000053c8       $N00084                    000000018000e3c8     windowsaccessbridge-64.exp
 0002:000053e8       $N00085                    000000018000e3e8     windowsaccessbridge-64.exp
 0002:0000540c       $N00086                    000000018000e40c     windowsaccessbridge-64.exp
 0002:00005425       $N00087                    000000018000e425     windowsaccessbridge-64.exp
 0002:00005439       $N00088                    000000018000e439     windowsaccessbridge-64.exp
 0002:00005452       $N00089                    000000018000e452     windowsaccessbridge-64.exp
 0002:00005471       $N00090                    000000018000e471     windowsaccessbridge-64.exp
 0002:00005489       $N00091                    000000018000e489     windowsaccessbridge-64.exp
 0002:000054a6       $N00092                    000000018000e4a6     windowsaccessbridge-64.exp
 0002:000054bf       $N00093                    000000018000e4bf     windowsaccessbridge-64.exp
 0002:000054dd       $N00094                    000000018000e4dd     windowsaccessbridge-64.exp
 0002:000054f5       $N00095                    000000018000e4f5     windowsaccessbridge-64.exp
 0002:0000550e       $N00096                    000000018000e50e     windowsaccessbridge-64.exp
 0002:0000552d       $N00097                    000000018000e52d     windowsaccessbridge-64.exp
 0002:000058dc       .idata$6                   000000018000e8dc     kernel32:KERNEL32.dll
 0002:00005998       .idata$6                   000000018000e998     user32:USER32.dll
 0002:00005a38       .idata$6                   000000018000ea38     vcruntime:VCRUNTIME140.dll
 0002:00005ba2       .idata$6                   000000018000eba2     ucrt:api-ms-win-crt-string-l1-1-0.dll
 0002:00005bc4       .idata$6                   000000018000ebc4     ucrt:api-ms-win-crt-stdio-l1-1-0.dll
 0002:00005be4       .idata$6                   000000018000ebe4     ucrt:api-ms-win-crt-environment-l1-1-0.dll
 0002:00005c0a       .idata$6                   000000018000ec0a     ucrt:api-ms-win-crt-heap-l1-1-0.dll
 0002:00005c2a       .idata$6                   000000018000ec2a     ucrt:api-ms-win-crt-runtime-l1-1-0.dll
 0003:000000e8       logFP                      000000018000f0e8     AccessBridgeDebug.obj
 0003:0000013c       ?__proc_attached@@3HA      000000018000f13c     MSVCRT:dll_dllmain.obj
 0003:00000140       GS_ExceptionRecord         000000018000f140     MSVCRT:gs_report.obj
 0003:000001e0       GS_ContextRecord           000000018000f1e0     MSVCRT:gs_report.obj
 0003:000006d8       ?is_initialized_as_dll@@3_NA 000000018000f6d8     MSVCRT:utility.obj
 0003:000006d9       ?module_local_atexit_table_initialized@@3_NA 000000018000f6d9     MSVCRT:utility.obj
 0003:000006e0       ?module_local_atexit_table@@3U_onexit_table_t@@A 000000018000f6e0     MSVCRT:utility.obj
 0003:000006f8       ?module_local_at_quick_exit_table@@3U_onexit_table_t@@A 000000018000f6f8     MSVCRT:utility.obj
 0005:00000120       $R000000                   0000000180011120     windowsaccessbridge-64.dll.res
 0005:00000530       $R000410                   0000000180011530     windowsaccessbridge-64.dll.res
 0005:00000748       $R000628                   0000000180011748     windowsaccessbridge-64.dll.res
